:100000000C94F6060C941E070C941E070C941E0705
:100010000C941E070C941E070C941E070C941E07CC
:100020000C941E070C9422090C94B1320C942C33BE
:100030000C941E070C941E070C941E070C941E07AC
:100040000C940C0E0C941E070C941E070C941E07A7
:100050000C941E070C941E070C941E070C94D429B4
:100060000C941E070C94CE2E0C94092F0C941E0792
:100070000C941E070C941E070C941E070C941E076C
:100080000C941E070C941E070C941E070C941E075C
:100090000C941E070C941E070C941E070C941E074C
:1000A0000C941E070C941E070C941E074E1D551D24
:1000B000551D4E1D551D551D551D551D551D551DB7
:1000C000551D551D551D551D551D551D551DBD1C39
:1000D000551D551D551D551D551D201C551D551DC6
:1000E000551D551D551D551D551D551D551D551D80
:1000F000551D551D551D551D551DC91CC91CC91C17
:10010000C91CC91CC91CC91CC91CC91C551D551DAD
:10011000551D551D551D551D251CC81CC81CC81C2A
:10012000C81C551DDF1CE71CEF1CF71CFF1C071D1E
:100130000F1D171D211D2B1D351D3F1D6C1C2C1C5B
:10014000551D551D551D551DBD1C551D551D551DB8
:10015000551D551D551D551D551DC71CC71CC71CBC
:10016000C71C551DDF1CE71CEF1CF71CFF1C071DDF
:100170000F1D171D211D2B1D351D3F1D6C1C2C1C1B
:10018000551D551D551D551DBD1C456E74657220B0
:100190006D656E752E2E2E00546F67676C6564203A
:1001A0006D6963726F50504D00546F67676C656482
:1001B00020696E7665727465642050504D2100543C
:1001C0006F67676C6564205458206D7574696E673D
:1001D0002100546F67676C65642074656C656D659C
:1001E000747279210050726F746F636F6C20657246
:1001F000726F7220776974682052580054696D6577
:100200006F7574207768656E20636F6E6E656374BA
:10021000696E6720746F20525800507265737320A6
:10022000616E79206B657920746F2063616E636500
:100230006C00436F6E6E656374696E6720746F2027
:1002400052582C20706F7765722075702074686525
:100250002052582028776974682062696E64207083
:100260006C7567206966206E6F74207573696E67A0
:1002700020616C776179732062696E642900546F24
:1002800067676C65642027696D6D65646961746575
:10029000206F75747075742700546F67676C6564A0
:1002A0002027736C617665206D6F64652700546F3D
:1002B00067676C65642027616C7761797320626978
:1002C0006E642700546F67676C65642050504D2042
:1002D0006368616E6E656C206C696D69740053654E
:1002E00074205253534920696E6A656374696F6E56
:1002F000206368616E6E656C2028303D3D646973D3
:1003000061626C6529005365742050504D206D6901
:100310006E696D756D2073796E630053657420622C
:100320006561636F6E20696E74657276616C0053EF
:10033000657420626561636F6E2064656C6179002D
:1003400053657420626561636F6E206672657175B6
:10035000656E637920696E20487A3A20303D646981
:100360007361626C652C2050783D504D522063685B
:10037000616E6E656C20782C2046783D4652532085
:100380006368616E6E656C20780053657420505709
:100390004D2073746F702064656C61792028302063
:1003A00064697361626C65642C20312D32353520AF
:1003B0003D3D20302E3173202D2035306D696E2962
:1003C000005365742050504D2073746F7020646525
:1003D0006C61792028302064697361626C65642CDB
:1003E00020312D323535203D3D20302E3173202DEA
:1003F0002035306D696E2900536574206661696C23
:10040000736166652064656C6179202830206469B9
:100410007361626C65642C20312D323535203D3D91
:1004200020302E3173202D2035306D696E29002A41
:100430002A2A2A2A2A2A2A2A2A2A2A2A2A2A2A2A1C
:100440002A2A2A2A2A2A2A2A2A2A2A2A00525820EA
:1004500041636B6564202D2072657665727420732C
:1004600075636365737366756C21002A2A2A2A2ACC
:100470002A2A2A2A2A2A2A2A2A2A2A2A2A2A2A2ADC
:100480002A2A2A2A2A2A2A2A002A2A2A2A2A2A2AF6
:100490002A2A2A2A2A2A2A2A2A2A2A2A2A2A2A2ABC
:1004A0002A2A2A2A2A2A0052582041636B6564208E
:1004B0002D20757064617465207375636365737353
:1004C00066756C21002A2A2A2A2A2A2A2A2A2A2AF6
:1004D0002A2A2A2A2A2A2A2A2A2A2A2A2A2A2A2A7C
:1004E0002A2A0056616C69642063686F69636573CA
:1004F000206172653A205B315D2D5B31365D2028CD
:100500006368616E6E656C20312D3136290053654C
:1005100074206F757470757420666F7220706F72BE
:100520007420005B585D2061626F727420636861A3
:100530006E67657320616E64206578697420525817
:1005400020636F6E666967005B535D20736176653B
:100550002073657474696E677320746F205258003D
:100560005B525D2072657665727420525820736507
:100570007474696E677320746F2064656661756C4E
:10058000747300557365206E756D62657273205BC0
:10059000312D445D20746F206564697420706F7222
:1005A0007473205B452D515D20666F7220736574F6
:1005B00074696E677300202D2072656365697665C6
:1005C0007220636F6E666967757261746F722C203A
:1005D000727820737720000A0A6F70656E4C525350
:1005E0006E6720005365742073657269616C2062C8
:1005F000617564726174653A200056616C696420AB
:1006000063686F696365733A2031202D20342B3481
:10061000202F2032202D2038202F2033202D20384D
:100620002B34202F2034202D203132202F20352034
:100630002D2031322B34202F2036202D2031360032
:10064000536574204368616E6E656C20636F6E66DF
:1006500069673A2000536574204461746172617463
:10066000652028302D32293A200053657420486FC8
:1006700070206368616E6E656C7320286D617820F0
:1006800032342C2073657061726174656420627904
:1006900020636F6D6D6173292076616C69642076CB
:1006A000616C75657320312D3235353A2000536504
:1006B00074206368616E6E656C2073706163696E2F
:1006C0006720287831306B487A293A2000536574C6
:1006D00020524620706F7765722028302D37293AD6
:1006E0002000536574205246206D6167696320289D
:1006F0006865782920652E672E203078444541446E
:10070000463030443A20005365742062617365209E
:100710006672657175656E63792028696E20487A06
:10072000293A20005B5A5D20656E746572207265FF
:1007300063656976657220636F6E6669677572615D
:1007400074696F6E207574696C79005B465D206416
:100750006973706C61792061637475616C20667275
:10076000657175656E636965732075736564005B9B
:10077000525D2063616C63756C6174652072616E9B
:10078000646F6D206B657920616E6420686F7020E6
:100790006C697374005B495D207265696E69746988
:1007A000616C697A652073657474696E677320740F
:1007B0006F20736B657463682064656661756C7423
:1007C00073005B585D2072657665727420636861A2
:1007D0006E67657320616E642065786974206D654D
:1007E0006E75005B535D207361766520736574746C
:1007F000696E677320746F20454550524F4D2061DC
:100800006E642065786974206D656E75005573653A
:10081000206E756D62657273205B302D395D2074BA
:100820006F206564697420706172616D65746572B2
:100830007300202D2053797374656D20636F6E668D
:10084000696775726174696F6E000A0A6F70656E10
:100850004C52536E6720005129204F757470757487
:10086000206265666F7265206C696E6B20283D465C
:100870005329203A2000502920536C617665206D61
:100880006F646520286578706572696D656E746146
:100890006C293A20004F292054696D656420424933
:1008A0004E44206174207374617274757020203A14
:1008B00020004E292050504D206F757470757420A3
:1008C0006C696D6974656420202020203A20004402
:1008D000495341424C4544004D292050504D20522F
:1008E00053534920746F206368616E6E656C2020DD
:1008F00020203A20004C292050504D206D696E690F
:100900006D756D2073796E63202875732920203AE8
:10091000200044495341424C4544004B2920466144
:10092000696C7361666520626561636F6E20696ED4
:1009300074762E2028312D32353573293A20004A1D
:1009400029204661696C7361666520626561636F29
:100950006E2064656C61792028302D323535203D5C
:100960003E20313073202D203135306D696E293AAB
:1009700020004929204661696C73616665206265C3
:1009800061636F6E206672712E203A200048292024
:1009900050574D2073746F702064656C617920200E
:1009A00020202020203A200047292050504D20733D
:1009B000746F702064656C617920202020202020D5
:1009C0003A20004629204661696C7361666520649F
:1009D000656C6179202020202020203A200050578B
:1009E0004D206368616E6E656C200066756E637481
:1009F000696F6E3A20002920706F72742000445491
:100A000046205548462033322D62697420313063C8
:100A100068004F70656E4C52536E675258206D6976
:100A20006E6920342F36636800466C7974726F6E7D
:100A30002F4F72616E6765525820554846203863C3
:100A40006800525820747970653A200044697361D7
:100A5000626C656400487A00203D3D200043616C73
:100A600063756C61746564207061636B6574206983
:100A70006E74657276616C3A20004229204D69637C
:100A8000726F202868616C66292050504D2020200C
:100A9000203A00412920496E7665727465642050C1
:100AA000504D20696E20202020203A003029204D12
:100AB0007574652062757A7A657220286D6F73741B
:100AC0006C79293A0039292053657269616C20627A
:100AD000617564726174653A00736D617274506F10
:100AE0007274004672536B79005472616E73706158
:100AF00072656E740044697361626C6564003829C4
:100B00002054656C656D657472793A202020202030
:100B10002020003729204368616E6E656C20636F6A
:100B20006E6669673A20200036292044617461723C
:100B30006174652028302D32293A20202000352983
:100B400020486F70206368616E6E656C733A202078
:100B5000202020003429204368616E6E656C20736C
:100B6000706163696E673A20200033292052462065
:100B7000706F7765722028302D37293A20202000A9
:100B80003229205246206D616769633A2020202077
:100B900020202020200031292042617365206672C8
:100BA000657175656E63793A2020200000000000B1
:100BB000240027002A002D0030000000000025003E
:100BC00028002B002E00310000000000230026002A
:100BD00029002C002F00040404040403040502026D
:100BE00002020403020202020606060606060404C6
:100BF00002020204040802011040804010204080DC
:100C00004080080204018040201002011080102062
:100C100040400000000200080E0000030401000B29
:100C200000000000000000000000000000000000C4
:100C3000070605040100080A0B0C0D09080B000249
:100C40000202010009040000010202000005240064
:100C500010010524010101042402060524060001F7
:100C60000705810310004009040100020A0000008A
:100C7000070502024000000705830240000004034C
:100C800009042203410072006400750069006E00CF
:100C90006F0020004C0065006F006E006100720064
:100CA00064006F0018034100720064007500690061
:100CB0006E006F0020004C004C0043001201000247
:100CC00000000040412336800001010200011201B2
:100CD00000020200004041233680000101020001B1
:100CE00000C18081C105010902A1010901A100859E
:100CF00001050919012903150025019503750181D5
:100D0000029501750581030501093009310938157E
:100D100081257F750895038106C0C005010906A1DC
:100D2000018502050719E029E715002501750195E0
:100D3000088102950175088103950675081500253F
:100D4000650507190029658100C009040200010337
:100D5000000000092101010001226500070584034C
:100D600040000100000000000000002A2B280000C5
:100D70000000000000000000000000000000000073
:100D80000000002C9EB4A0A1A2A434A6A7A5AE3654
:100D90002D3738271E1F20212223242526B333B6C2
:100DA0002EB7B89F8485868788898A8B8C8D8E8F95
:100DB000909192939495969798999A9B9C9D2F3198
:100DC00030A3AD350405060708090A0B0C0D0E0FFC
:100DD000101112131415161718191A1B1C1DAFB178
:100DE000B0B50000072CC230FD319A3411241FBE6B
:100DF000CFEFDAE0DEBFCDBF14E0A0E0B1E0E8ED78
:100E0000FCE602C005900D92A432B107D9F717E0B5
:100E1000A4E2B4E001C01D92A233B107E1F71DE0E6
:100E2000CCEEDDE004C02297FE010E942436C43ED1
:100E3000D107C9F70E9407310C946A360C94000060
:100E4000A0E0B0E0E6E2F7E00C943B36EC01A880CD
:100E5000B980CA80DB80A114B104C104D10441F47B
:100E600084E2A82E89EDB82E8BE5C82E87E0D82E17
:100E7000C601B5012DE133EF41E050E00E94F335AA
:100E800027EA31E440E050E00E949F357B018C016D
:100E9000C601B5012DE133EF41E050E00E94F3358A
:100EA000CA01B9012CEE34EF4FEF5FEF0E949F357E
:100EB0006E0D7F1D801F911F97FF04C06150704011
:100EC00080409048688379838A839B839B01AC012F
:100ED0005F77B901CA01CDB7DEB7EAE00C945736A7
:100EE0000E942007089584E193E00E94200708955E
:100EF0006093140370931503809316039093170364
:100F00000895A0E0B0E0E7E8F7E00C943436EC0197
:100F10002B016A016115710519F0FB019183808332
:100F2000C114D10449F0C6010297839728F020E04C
:100F300030E040E050E0DCC0A9908A2D90E00E94B3
:100F40002836892BC9F7FDE2AF1621F4A990332486
:100F5000339405C08BE2A81609F4A9903324C11478
:100F6000D10421F0E0E1CE16D10411F5F0E3AF1683
:100F700069F48881883711F0883541F4A980229678
:100F800082E0382A20E1C22ED12C12C0C114D10433
:100F900079F4E0E3AE1659F199E9E92E99E9F92ED1
:100FA00099E9092F99E1192F8AE0C82ED12C3AC06E
:100FB000FAE0CF16D10491F080E1C816D10429F0EF
:100FC000E8E0CE16D104F9F415C0BFEFEB2EBFEF69
:100FD000FB2EBFEF0B2FBFE01B2F24C0A9E9EA2E89
:100FE000A9E9FA2EA9E90A2FA9E11A2F1BC0F8E0F6
:100FF000CF2ED12CEFEFEE2EEFEFFE2EEFEF0E2FD8
:10100000EFE11E2F0FC09601442737FD4095542F66
:101010006FEF7FEF8FEF9FEF0E94D135C901DA01AB
:101020007C018D0120E030E040E050E060E03601DE
:10103000882477FC8094982C70EDB72EBA0CF9E0D8
:10104000FB1570F48A2D81548A3118F499ECB92E6D
:1010500006C08A2D81568A3148F589EAB82EBA0C25
:101060008B2D90E08C159D050CF56F3FE9F0E21695
:10107000F30604071507B8F0CA01B901A4019301EA
:101080000E949F359B01AC018B2D90E0A0E0B0E069
:10109000280F391F4A1F5B1F281739074A075B07AC
:1010A00010F061E001C06FEFA990C6CF4114510468
:1010B00051F0662311F0219703C031FE04C022973E
:1010C000F201D183C08330FE07C050954095309522
:1010D00021953F4F4F4F5F4F67FF0AC082E290E07C
:1010E00090933107809330072FEF3FEF4FEF5FEF83
:1010F000B901CA01CDB7DEB7E1E10C945036FC016D
:1011000088279927E89421912032E9F3293010F0BB
:101110002E30C8F32B3241F02D3239F4689404C0DC
:101120000E94D408820F911D219120532A30C0F3D0
:101130001EF4909581959F4F089544E254E00E94DB
:10114000A2080895009731F4DA018D919C910097DF
:1011500009F40EC0DC01FB013D912191222319F01D
:101160003217C9F3FACF332331F4DA011D921C92FE
:101170008827992708951197AF93BF93FB013D915D
:101180002191321771F4332321F48827992711977D
:1011900002C01E921196FA01A193B0839F918F9184
:1011A0000895222369F7EACF7AE0979F902D879FD1
:1011B000802D910D1124089580912604813019F419
:1011C00082E08093260480912604833019F484E021
:1011D000809326040895009721F19C0140E050E09F
:1011E00068E478EE81E090E00E94F335C901DA010D
:1011F0008F3F9105A105B10531F028F08FEF90E008
:10120000A0E0B0E008C00097A105B10521F481E09D
:1012100090E0A0E0B0E08093D1008091C0008061B8
:1012200003C08091C0008F7E8093C0000895EBE6DC
:10123000F0E0808180688083E8E6F0E08081816072
:10124000808308951F920F920FB60F9211242F934F
:101250003F934F935F936F937F938F939F93AF933E
:10126000BF93EF93FF931F9902C00E94DC08FF9188
:10127000EF91BF91AF919F918F917F916F915F910E
:101280004F913F912F910F900FBE0F901F90189587
:1012900081E008951F93182F0E9448098823E9F0E0
:1012A0002FB781E080931406F89480910008909104
:1012B00001088757974709F0A89588E18093600057
:1012C00010936000112341F0809100089091010873
:1012D0008757974709F0A8952FBF1F9108958091D0
:1012E0005004E82FF0E03496DF0126E0AA0FBB1F80
:1012F0002A95E1F720E030E040E050E060E070E067
:10130000F999FECFCB018A0F9B1F92BD81BDF89A40
:1013100080B5542F432F322F2227280F311D411D16
:10132000511D6F5F7F4F6430710551F72E513E4B59
:10133000414C5E4D19F020E030E01FC09F0186E077
:10134000220F331F8A95E1F72C5F3F4FE7E2F4E06D
:10135000F999FECF32BD21BDF89A80B581932F5FF8
:101360003F4F84E0E035F80799F720E030E08091C6
:101370002704893011F421E030E0C901089589E0A3
:101380008093270480E092ECA1E0B0E080932804F1
:1013900090932904A0932A04B0932B0487E08093B0
:1013A000340480EC92E9ADEEB9E180932C04909383
:1013B0002D04A0932E04B0932F0485E08093350470
:1013C0008DEE9EEFADEABEED809330049093310434
:1013D000A0933204B0933304A6E3B4E080E090E03D
:1013E000863010F0E0E004C0FC01E351FC4FE081E6
:1013F000ED9301968831910599F782E080934E0430
:101400008AE080934F0408958436910520F4BC014E
:1014100080E090E025C08E3B910550F48A559040C5
:10142000BC0180E090E02AE030E040E050E016C0EF
:10143000823D910550F4845B9040BC0180E090E0D7
:1014400024E630E040E050E009C08D5C9040BC01F3
:1014500080E090E028E532E040E050E00E949F35D7
:1014600024E630E040E050E00E949F35089590E08F
:101470008C599F4F0E94040A0895DC019896EC91C4
:10148000F0E0E770F070EB51FC4F808108958F928F
:101490009F92AF92BF92CF92DF92EF92FF920F9303
:1014A0001F938C010E943D0AD80197962C9130E041
:1014B00043E150E0249FF001259FF00D349FF00D93
:1014C0001124E85EFC4F80809180A280B38090E080
:1014D0000F96AA2797FDA095BA2FBC01CD0120E455
:1014E0003FE14DE750E00E949F35A50194010E9425
:1014F000D13569017A0180ED97E0A0E0B0E0C80E37
:10150000D91EEA1EFB1ED80198968C91887181F035
:1015100060E07EEE8AEB9BE0A50194010E94D1354C
:1015200028513C4F4F4F5F4FC20ED31EE41EF51E95
:1015300087EE93E0A0E0B0E0C80ED91EEA1EFB1EC5
:10154000C701B60128EE33E040E050E00E94D135FB
:10155000CA01B90128EE33E040E050E00E949F3517
:101560001F910F91FF90EF90DF90CF90BF90AF90C1
:101570009F908F9008958F3F910509F010F480E0BF
:10158000089522E08030920710F481E008958050A1
:10159000934010F083E0089582E00895CF92DF92A7
:1015A000FF920F931F93CF93DF93F82FEB016A0104
:1015B000182F1695E0E088819981D6018C938A8155
:1015C0009B8111968C9311978C819D8112968C939F
:1015D00012978E819F8113968C931397288139815E
:1015E0004A815B816C817D818E819F819295990F6B
:1015F000990F907C832F8370982B852F8370880F91
:10160000880F982B872F83708295807F982B149654
:101610009C9385E090E0C80ED91E2896EF5F1E17B8
:1016200050F6F0FF21C0888199810E94BB0AF82EF4
:101630008A819B810E94BB0A182F8C819D810E9408
:10164000BB0A082F8E819F810E94BB0AF294FF0C77
:10165000FF0C50ECF5221295107F1F29182B000F5C
:10166000000F012BD6010C93DF91CF911F910F91A9
:10167000FF90DF90CF90089523E08032920718F416
:1016800020E030E026C023E0883E920748F49C0129
:101690002F513340F4E036952795FA95E1F719C0BC
:1016A00027E0803D920720F49C012C5D334011C05F
:1016B00028E08839920718F02FEF33E00AC09C0128
:1016C000285C3740E4E036952795EA95E1F72D5000
:1016D0003C4FC90108959C013695279525753575B0
:1016E000821B930B9C01369527953695279523737E
:1016F000337383739373280F391FC90144E09695A0
:1017000087954A95E1F7820F931F8F709F7021E0B4
:1017100031E0AC01429FC001439F900D529F900D5C
:101720001124892F0895382F20E08091A6059091EB
:10173000A7058227932740E061E270E19C01220F18
:10174000331F97FF04C0C9018627972701C0C9012D
:101750004F5F483099F79093A7058093A6050895A9
:10176000882339F0299800002A9A0000299A00005D
:101770000895299800002A980000299A00000895E9
:10178000299A000083B12998000090E0F3E0969533
:101790008795FA95E1F7817008950F931F93082FAD
:1017A0005E9A29985E9810E0802F80780E94B00B96
:1017B000000F1F5F1830C1F729981F910F910895EE
:1017C0008F770E94CD0B08950F931F93082F10E081
:1017D000802F80780E94B00B000F1F5F1830C1F778
:1017E00029981F910F9108950F931F93299880E0D6
:1017F00000E0182F110F0E94C00B810F0F5F0830FF
:10180000C1F71F910F9108950E94E00B0E94F40B05
:101810005E9A08951F93162F80680E94CD0B812F2A
:101820000E94E40B5E9A1F9108951F93109130045B
:101830001827E7E2F4E0E80FF11D89E767850E94C9
:101840000A0C8DE3612F0E940A0C82E4612F0E9432
:101850000A0C1F91089586E20E94040C08950F93CC
:101860001F938C018CE1F80164810E940A0C8DE1C8
:10187000F80165810E940A0C8EE1F80166810E94E0
:101880000A0C80E2F80167810E940A0C81E2F801EB
:1018900060850E940A0C82E2F80161850E940A0CB0
:1018A00083E2F80162850E940A0C84E2F8016385F4
:1018B0000E940A0C85E2F80164850E940A0C8AE203
:1018C000F80165850E940A0C8EE6F80166850E9483
:1018D0000A0C8FE6F80167850E940A0C80E7F80180
:1018E00060890E940A0C81E7F80161890E940A0C54
:1018F00082E7F80162890E940A0C1F910F910895F6
:10190000EF92FF920F931F93CF93DF937B018C0194
:10191000603028E372072CE982072CE1920728F552
:1019200020E836E948E950E00E94D135E90168979E
:10193000B90180E090E020E839E647E65FEF0E94D9
:101940009F356E0D7F1D801F911F02E0660F771F70
:10195000881F991F0A95D1F721E732E040E050E057
:101960000E94D135890180E421C020E03DE241E3BD
:1019700051E00E94D135E9016897B90180E090E01B
:1019800020E033ED4EEC5EEF0E949F356E0D7F1D23
:10199000801F911F660F771F881F991F21E732E074
:1019A00040E050E00E94D135890180E69E012F7110
:1019B000622F680F85E70E940A0C86E7612F0E945C
:1019C0000A0C87E7602F0E940A0CDF91CF911F91CC
:1019D0000F91FF90EF9008959F92AF92BF92CF9298
:1019E000DF920F93DF93CF9300D000D0CDB7DEB757
:1019F000982E83E00E94040C80936C0484E00E9483
:101A0000040C80936D0486E060E00E940A0C87E07D
:101A100061E00E940A0C89E06FE70E940A0C8AE0EC
:101A200065E00E940A0C8BE065E10E940A0C8CE0E4
:101A300062E10E940A0C8DE06DEF0E940A0C8EE0BC
:101A400060E00E940A0C992019F087E793E008C033
:101A500080914E0423E1829FC0011124885E9C4F37
:101A60000E942F0C80E36CE80E940A0C82E36FE076
:101A70000E940A0C83E362E40E940A0C84E36AE099
:101A80000E940A0C85E36AE20E940A0C86E36DE27A
:101A90000E940A0C87E364ED0E940A0C88E360E070
:101AA0000E940A0C89E360E00E940A0C992049F028
:101AB0002EE1A22E2EEBB22E21ECC22E2EEDD22E36
:101AC00008C0A0903004B0903104C0903204D0908F
:101AD00033040AE38D2D9927AA27BB2789839A838C
:101AE000AB83BC83802F69810E940A0C802F8B5F9F
:101AF00069810E940A0CDC2CCB2CBA2CAA240F5F23
:101B00000E3341F783E46FEF0E940A0C84E46FEF19
:101B10000E940A0C85E46FEF0E940A0C86E46FEFC6
:101B20000E940A0C992019F08DE666E003C08DE64C
:101B3000609134040E940A0C89E760E00E940A0C5C
:101B40008AE7609135040E940A0C83E760E00E94F6
:101B50000A0C84E760E00E940A0C992029F060ECEE
:101B600072E98DEE99E108C060912C0470912D040A
:101B700080912E0490912F040E94800C0F900F9062
:101B80000F900F90CF91DF910F91DF90CF90BF908A
:101B9000AF909F90089587E061E00E940A0C8EE765
:101BA00064E20E940A0C88E063E00E940A0C88E06C
:101BB00060E00E940A0C87E065E00E940A0C85E064
:101BC00062E00E940A0C83E00E94040C80936C0483
:101BD00084E00E94040C80936D040895582F409176
:101BE0001105842F90E0FC01EF70F0709F012F5FD2
:101BF0003F4F64E0959587956A95E1F72817390777
:101C000051F0EF5FFA4F5083842F8F5F8F70407FCA
:101C1000842B8093110508951F920F920FB60F9297
:101C200011241F932F933F934F935F936F937F9351
:101C30008F939F93AF93BF93CF93DF93EF93FF93D4
:101C4000C0918600D09187002091530530915405B2
:101C500080913205882309F047C0CE01821B930B87
:101C60009C0180914F0487FD02C03695279599E02D
:101C7000253C390708F18091AA038630D0F0809185
:101C8000AA038F3FB1F020E00EC0E22FF0E0EE0F8C
:101C9000FF1FDF01AD5CBA4F8D919C91E657FC4F61
:101CA000918380832F5F8091AA03281770F310928D
:101CB00031051092AA0318C082E02D3B380760F16D
:101CC0008091AA03803140F51091AA03C9010E94B6
:101CD0003C0BE12FF0E0EE0FFF1FED5CFA4F91831C
:101CE00080831F5F1093AA03D0935405C0935305BC
:101CF000FF91EF91DF91CF91BF91AF919F918F9124
:101D00007F916F915F914F913F912F911F910F9014
:101D10000FBE0F901F9018958FEF8093AA03E4CF0A
:101D200083E0809380008AE98093810080914F0452
:101D300086FD05C0809181008064809381008FEFD3
:101D40009FEF909389008093880080916F0080625C
:101D500080936F0008956F3020F0869586958054AB
:101D600008958DE0689F802D11240895982F80910B
:101D70009F05882311F481E003C0813021F482E0C3
:101D800080939F050895803190F5E82FF0E0ED5C99
:101D9000FA4F90838F5F80939F05803151F520919A
:101DA0003205A5E3B5E0213039F41196EC91119795
:101DB000E695E6958C9109C08D919C911197E92F3C
:101DC000E695E695E69596958795E03140F4F0E046
:101DD00090E0EE0FFF1FE657FC4F91838083109237
:101DE0003105129685E0A334B807E9F608951092FC
:101DF0009F0508950F931F93CF93DF9390919F05B5
:101E0000992339F48F3009F002C181E080939F0556
:101E1000FEC0983148F4E92FF0E0EE5CFA4F808381
:101E20009F5F90939F05F3C0983109F0EEC088231F
:101E300009F0EBC0C0E0D0E00BE010E0DE0163E0B1
:101E4000AA0FBB1F6A95E1F7C09FB001C19F700D3B
:101E5000D09F700D1124FB01ED5CFA4F8081218130
:101E6000922F977095958795FD01EE0FFF1FE6570E
:101E7000FC4F91838083FB01EC5CFA4F30813695F7
:101E8000369536952181422F4295440F407E842F0E
:101E9000832B269526952695922F97709595879555
:101EA000FD01EE0FFF1FE457FC4F91838083FB0180
:101EB000EB5CFA4F8081829586958695837041818F
:101EC000942F990F990F292F282B429546954695C7
:101ED000437082818170880F880F382F342B35959D
:101EE0002795FD01EE0FFF1FE257FC4F3183208342
:101EF000FB01E95CFA4F308136952181422F4795ED
:101F000044274795842F832B2695922F977095957C
:101F10008795FD01EE0FFF1FE057FC4F91838083F3
:101F2000FB01E85CFA4F308132953F702181422FEE
:101F30004295407F842F832B22952F70922F97708C
:101F400095958795FD01EE0FFF1FEE56FC4F91838F
:101F50008083FB01E75CFA4F8081881F8827881FF8
:101F60004181942F990F292F282B441F4427441F68
:101F700082818370880F382F342B35952795FD018A
:101F8000EE0FFF1FEC56FC4F31832083FB01E55C15
:101F9000FA4F3081369536952181422F4295440F74
:101FA000440F407C842F832B26952695922F977083
:101FB00095958795AA0FBB1FFD01EA56FC4F9183AB
:101FC0008083645C7A4FFB012081229526952770DF
:101FD0004181342F330F330F330F832F822B942FF4
:101FE00092959695977095958795A856BC4F1196A2
:101FF0009C938E932196C230D10509F01FCF80911A
:10200000490583FD02C01092310510929F05DF91B2
:10201000CF911F910F910895DF92EF92FF920F934E
:102020001F93CF93DF93682F40919F05442359F46A
:10203000883AB1F41092A7051092A60588EA0E948A
:10204000930B81E06FC0413019F48093A40504C064
:10205000423031F48093A505862F0E94930B5DC01A
:102060007091A505272F30E0220F331FE42FF0E0F9
:10207000C90102968E179F0734F0433268F7E05D7E
:10208000FA4F6083E9CF2D5F3F4F4091A6055091F5
:10209000A705E217F30749F4962F80E04827592750
:1020A0005093A7054093A60538C0862F90E04817A7
:1020B000590789F58091A405813069F5713118F0CF
:1020C00080E18093A505D090A505F3E3EF2EF5E020
:1020D000FF2E00E010E01BC0F701D081C0E081813D
:1020E00090E08C2B9D2BE3E096958795EA95E1F7A0
:1020F0000E943C0BF801EE0FFF1FE657FC4F918347
:1021000080830F5F1F4F82E090E0E80EF91E0D15EF
:1021100018F31092310510929F0580919F05882336
:1021200019F08F5F80939F05DF91CF911F910F91E1
:10213000FF90EF90DF900895882319F460E071E03C
:1021400002C063E071E082E696E00E94B92E089535
:10215000CF92DF92EF92FF921F93182F0E942A2AAC
:102160009B01AC018091A0059091A105A091A205D1
:10217000B091A30569017A01C81AD90AEA0AFB0AD3
:10218000D701C60189589341A040B04010F0109289
:102190009F052093A0053093A1054093A20550937D
:1021A000A30590913205892F8150823020F4812F30
:1021B0000E94B60E0BC0933021F4812F0E94FA0EBC
:1021C00005C0943019F4812F0E940C101F91FF90CC
:1021D000EF90DF90CF900895FF920F931F93CF93CE
:1021E000DF93182F092FF62E8EE30E940A0C212F61
:1021F000302FC901EC0110E005C08FE769910E9402
:102200000A0C1F5F1F15C8F385E064E00E940A0CEA
:1022100083E00E94040C80936C0484E00E94040C10
:1022200080936D040E942A2A60936E0470936F0459
:10223000809370049093710487E069E00E940A0C17
:1022400081E080932604DF91CF911F910F91FF9041
:1022500008950E94EC10809126048130D9F40E94E8
:102260002A2A20916E0430916F044091700450919D
:102270007104621B730B840B950B605A7648814086
:10228000904040F4E8CF82E696E067E071E00E947B
:10229000B92E0895809126048130A9F3089588EF1E
:1022A00096E06EE70E9482300895BF92CF92DF924F
:1022B000EF92FF920F931F93CF93DF936C0188EF00
:1022C00096E06EE70E948230760100E010E0C0E008
:1022D000D0E080E2B82E0AC00830110521F49E013A
:1022E0002095F60120870894E11CF11CF70160811C
:1022F000862F8D57823040F488EF96E06DE70E947C
:102300008230F70160816B2588EF96E00E94823071
:102310000115110551F0F70180819E01280F311D33
:10232000C32FDD27C20FD31FD0700F5F1F4F09309F
:10233000110591F6DF91CF911F910F91FF90EF90D2
:10234000DF90CF90BF900895DF93CF93CDB7DEB7E6
:1023500029970FB6F894DEBF0FBECDBF382FE62FFA
:102360008091160590E0019664E270E00E94BE350F
:10237000982F8093160588E9898380E18A839130BC
:1023800071F0913028F0923099F09330E1F416C05A
:1023900085E08B8381EF8C832F5F2D8317C09B8318
:1023A00081EF8C8384E6489FC00111249D830EC079
:1023B00084E08B8381EF8C833D8308C09B8381EF16
:1023C0008C83ED8303C00E944F1104C0CE0101969F
:1023D0000E94551129960FB6F894DEBF0FBECDBFEF
:1023E000CF91DF9108950F931F93CF93DF93182F11
:1023F000092F88EF96E06EE70E948230212F302F60
:10240000C901EC0110E000E288818D57823040F470
:1024100088EF96E06DE70E9482308881802788836C
:1024200088EF96E069910E9482301F5F193061F752
:1024300088EF96E06EE70E948230DF91CF911F9186
:102440000F910895DF93CF93CDB7DEB729970FB6DD
:10245000F894DEBF0FBECDBF382F809116058823BC
:1024600079F48EEF89833A836B83842F90E095957E
:1024700087958C832D83198618861F821E822FC014
:1024800040911105842F90E09C012F70307054E032
:10249000959587955A95E1F78217930721F18DEF6E
:1024A00089831A821B82DE01149620E008C0EF5F48
:1024B000FA4F80818D93405F2F5F263069F0842F23
:1024C00090E0FC0134E0F595E7953A95E1F78F70DF
:1024D0009070E817F90759F7409311052A83CE0148
:1024E00001960E94F3118091160590E0019666E036
:1024F00070E00E94BE358093160529960FB6F894B9
:10250000DEBF0FBECDBFCF91DF9108959F92AF92F6
:10251000BF92CF92DF92EF92FF920F931F93B82E4C
:10252000A62ED42EC22E902E0E942A2A7B018C0128
:1025300080910005209112053091130540911405FA
:10254000509115058823B1F0D801C701821B930B68
:10255000A40BB50B815E9E42A040B04020F12C2D13
:10256000DC1408F42D2D8B2D6A2D422F292D0E946D
:10257000A41111C0D801C701821B930BA40BB50B8A
:1025800081539547A040B04070F08B2D6A2D4D2DA2
:102590002C2D0E942212E0921205F0921305009356
:1025A0001405109315051F910F91FF90EF90DF9088
:1025B000CF90BF90AF909F900895219A229A239830
:1025C0008BE060E00E94CC2A8CE061E00E94CC2A83
:1025D000089588E08093C1008AE061E00E94CC2ADF
:1025E0008AE060E00E94592B0895AF92BF92CF928B
:1025F000DF92EF92FF920F931F93DF93CF93CDB7AC
:10260000DEB76C970FB6F894DEBF0FBECDBF0E9449
:102610002A2A7B018C0181E00E94EC0CF4E7AF2EAA
:102620006E010894C11CD11CE3E0BE2EA982C60134
:1026300061E00E942911B09226040E94CB0D6AEF3E
:1026400070E080E090E00E94502A80912604833060
:1026500009F08AC082E696E00E94BD2B892B09F022
:1026600083C00E942A2A6E197F09800B910B605843
:10267000734C894C914008F077C0D8CF8FE70E9407
:10268000E00B0E94F40B843509F05CC089830E9442
:10269000F40B182F00E01093FF040093FE040E9437
:1026A000F40B080F111D1093FF040093FE040E9409
:1026B000F40B8093FD040E94F40B8093FC048131A1
:1026C00008F040C0FF2407C00E94F40B04521B4FC7
:1026D000F8018083F3940F2D10E08091FC0490E0CA
:1026E000880F991F0817190778F380E78983CE01AF
:1026F000019661E00E94291183E0809326040E94E4
:10270000CB0D62E370E080E090E00E94502A80915F
:1027100026048330A9F08FE70E94E00B0E94F40B9F
:10272000803581F4898301E514E00E94F40BF801FF
:1027300081938F01F4E00C361F07B9F781E003C0E5
:1027400082E001C083E06C960FB6F894DEBF0FBE46
:10275000CDBFCF91DF911F910F91FF90EF90DF9050
:10276000CF90BF90AF90089580912604833009F0F8
:1027700085CFE6CF83E00E94040C80936C0484E054
:102780000E94040C80936D0487E061E00E940A0CB3
:102790006AE070E080E090E00E94502A0E94CB0D39
:1027A000000008950F931F93082F17C05F9A64E6E7
:1027B00070E080E090E00E94502A5F9864E670E04C
:1027C00080E090E00E94502A1F5F101778F36CE2BF
:1027D00071E080E090E00E94502A10E0F6CF482F90
:1027E000392F25E00DC0F999FECF1FBA842F932F02
:1027F00092BD81BD60BD0FB6F894FA9AF99A0FBEEA
:10280000215059F0F999FECF842F932F92BD81BDAD
:10281000F89A80B5681739F7089582E00E94D213BC
:102820000895CF92DF92EF92FF920F931F93CF9371
:10283000DF93C0E0D0E008E110E08EE1C82E8EEB1F
:10284000D82E81ECE82E8EEDF82E8091500490E089
:102850000496B6E0880F991FBA95E1F7A701960193
:10286000002E04C056954795379527950A94D2F7C0
:102870008C0F9D1F622F0E94EF132196085010406D
:10288000C430D10511F7C0E0D0E08091500490E051
:10289000A6E0880F991FAA95E1F78C5F9E4FFE0175
:1028A000E95DFB4F8C0F9D1F60810E94EF13219605
:1028B000C932D10551F7DF91CF911F910F91FF9050
:1028C000EF90DF90CF90089580E490E06091500405
:1028D0000E94EF130895F999FECF80E490E092BD35
:1028E00081BDF89A80B580935004843020F0109216
:1028F00050040E94641408951F93182F0E946B14B3
:1029000080915004811731F0143020F4109350045A
:102910000E9464141F9108951F93182F0E942A2A61
:102920006093120570931305809314059093150519
:1029300010930005112329F440E855E260E070E0AF
:1029400004C040E051EE60E070E088EF96E00E9445
:10295000882F1F910895809118058130D1F0813022
:1029600020F0823009F043C037C082E10E948C2BF6
:10297000892B09F03CC081E0809318050E941C2A35
:102980006093190570931A0580931B0590931C059D
:10299000089582E10E948C2B892BD9F40E941C2A75
:1029A0002091190530911A0540911B0550911C0585
:1029B000621B730B840B950B695E734080409040E3
:1029C000B0F082E08093180580ED97E00E94EB085C
:1029D000089510921805089582E10E948C2B892B8E
:1029E00031F080E090E00E94EB0810921805089505
:1029F000AF92BF92CF92DF92EF92FF920F931F930D
:102A0000CF93DF938CE00E94040C8823B9F582E613
:102A100096E063E171E00E94B92E5F9A80E00E9427
:102A2000EC0C0E94CB0D5F9829C080913205882361
:102A300039F088EF96E00E9449300E94A8101EC02D
:102A400080919D05C82FD0E09E012F5F3F4F2F71D1
:102A5000307080919C0590E02817390779F088EF55
:102A600096E00E944930CD58DA4F888380919D05C9
:102A700090E001968F71907080939D0588EF96E0AD
:102A80000E940F30892B89F680912604843009F04A
:102A90008CC00E942A2A609321057093220580939E
:102AA000230590932405611571058105910561F455
:102AB00081E090E0A0E0B0E08093210590932205B2
:102AC000A0932305B093240580912D0590912E05A8
:102AD000816090932E0580932D0583E080932604DA
:102AE0008FE70E94E00BCAE6D5E00E94F40B8993C1
:102AF00005E0C337D007C9F74091550580916A05B5
:102B0000282F30E0842F90E08227932786FF40C053
:102B100080E4482740935505C90188739070C89791
:102B200009F510E014C01F5F80914F04E12FF0E021
:102B300084FF06C0E659FA4F80810E94EE0D07C05F
:102B4000E659FA4F88EF96E060810E948230212F8B
:102B500030E080916A0590E087709070821793074B
:102B600014F716C02F733070232B91F480916B05EE
:102B70008093250580916C058093270580916D05D4
:102B8000809328058091700580932F051092300561
:102B900080919E05813019F482E080939E0580919A
:102BA0009E05833011F410929E050E942A2A5B0133
:102BB0006C018091290590912A05A0912B05B09177
:102BC0002C050097A105B105C9F0A6019501281BA8
:102BD000390B4A0B5B0BDA01C901885B9B40A040B3
:102BE000B04060F00E942B0C8093260510922905BE
:102BF00010922A0510922B0510922C0587E294E082
:102C00000E94470A20911D0530911E0540911F0525
:102C10005091200586017501E21AF30A040B150B89
:102C2000E616F7060807190708F4F1C0A0921D057B
:102C3000B0921E05C0921F05D09220058091000819
:102C4000909101088757974709F0A8958091310521
:102C5000883008F0D4C0809131058F5F80933105B2
:102C6000E0902105F09022050091230510912405A4
:102C7000E114F1040105110511F187E294E00E94CD
:102C8000470AAE18BF08C00AD10A6A157B058C0531
:102C90009D0588F480914F0485FD04C080ED97E088
:102CA0000E94EB0810922105109222051092230534
:102CB0001092240504C080E090E00E94EB089091FF
:102CC0005505907C9093550500919D0510919C05AC
:102CD0000117B1F180919E05823091F59058909343
:102CE000550587E294E00E943D0A893010F048E0E3
:102CF00002C0482F415030E013C03F5FA32FB0E027
:102D0000812F90E0FC01ED58FA4F2081FD01EB5A34
:102D1000FA4F2083AD56BA4F2C930196182F1F718E
:102D2000341710F4101749F710939C05832F895C12
:102D300090915505892B80935505309393051AC0C2
:102D400020919E052430D1F490919305E4E9F5E0BB
:102D5000A6E5B5E0292F30E02E0F3F1F02C081917C
:102D60008D93E217F307D9F7995C80915505982B5D
:102D70009093550583E080939E0523C080911805AC
:102D8000823029F49160909355055F9A0FC090931B
:102D900055055F98222319F481E080939E05809168
:102DA0009E05833019F484E080939E05F894809109
:102DB0004F0487706AE873E046E555E00E94CE0A4A
:102DC0007894469A809117050E94150C87E294E04A
:102DD0000E943D0A682F85E595E00E94EC10E09185
:102DE0001705EF5FE0931705E83131F0F0E0E95D9A
:102DF000FB4F8785882359F41092170508C08091EE
:102E00003105883009F45F9A89E08093310580911B
:102E10004F04887171F180912604823051F58091C0
:102E20002D0590912E05880F991F90932E05809364
:102E30002D0583E0809326040E94CB0D0E942A2A50
:102E40006093290570932A0580932B0590932C0598
:102E5000611571058105910561F481E090E0A0E0C4
:102E6000B0E08093290590932A05A0932B05B09399
:102E70002C0580914F0484FF1EC080912D059091F8
:102E80002E058E7F0E946B0B182F80912505609177
:102E90002F050E94AB0E082F80912605612F0E94FE
:102EA000AB0E282F8091270560912805402F0091B7
:102EB00050040E94861246980E94AB14DF91CF9175
:102EC0001F910F91FF90EF90DF90CF90BF90AF9048
:102ED000089582E696E0609173040E941E2C089586
:102EE0001F93182F82E696E0612F0E941E2C80917E
:102EF00073048127809373041F9108951F93192FE2
:102F00000E947017812F0E9470171F910895DF9201
:102F1000EF92FF920F931F93D82E7B0110927304B0
:102F200002E616E0C80165EB0E941E2CC80162E6AD
:102F30000E941E2C8D2D0E947017C7010E947E17C3
:102F40001F910F91FF90EF90DF9008951092DA0497
:102F500085E6E5E7F4E0DF011D928A95E9F708953B
:102F60001F93182F8F3711F08830E1F5E091DA04C4
:102F7000EE2309F455C0E150E093DA04F0E0EB5899
:102F8000FB4F108282E696E06DE00E941E2C10E05E
:102F90000AC0E12FF0E0EB58FB4F82E696E060813B
:102FA0000E941E2C1F5F8091DA04181790F382E6AE
:102FB00096E060E20E941E2C82E696E06DE00E94A0
:102FC0001E2C10E00AC0E12FF0E0EB58FB4F82E628
:102FD00096E060810E941E2C1F5F8091DA04181712
:102FE00090F31CC08B3119F40E94A6171FC08D30BE
:102FF000E9F08A30D9F08091DA04843688F482E6E8
:1030000096E0612F0E941E2C8091DA04E82FF0E0F8
:10301000EB58FB4F10838F5F8093DA0480E007C08A
:1030200082E696E067E00E941F2DF8CF81E01F91B5
:1030300008951F93CF93DF93C6E3D4E010E03BC025
:1030400082E696E062E271E00E94B62E82E696E0A9
:10305000612F4AE050E00E942D2E82E696E06FE25A
:1030600071E00E94B62E699170E080E090E02091BE
:10307000350430E040E050E00E949F3520E137E227
:1030800040E050E00E949F35DC01CB0140912C04D0
:1030900050912D0460912E0470912F04480F591FF8
:1030A0006A1F7B1F82E696E02AE030E00E94F42D42
:1030B0001F5F183119F08881882311F6DF91CF91B5
:1030C0001F910895EF92FF920F931F93882339F475
:1030D00082E696E06CE47AE00E943D2D3BC090E0F1
:1030E0000E94040A24E630E040E050E00E94D1351E
:1030F000122F032FF42EE52E622F732F842F952F7E
:103100002AE030E040E050E00E94D13582E696E0CF
:10311000BA01A9012AE030E00E94E52D82E696E09E
:103120006EE20E941F2D612F702F8F2D9E2D2AE0A1
:1031300030E040E050E00E94D135AB01BC0182E6B6
:1031400096E02AE030E00E94E52D82E696E063E713
:103150000E94512D1F910F91FF90EF900895FF92C3
:103160000F931F93CF93DF9382E696E062E47AE0B9
:103170000E94FC2C80915104813041F482E696E05B
:1031800069E27AE00E943D2DFF2466C0823029F476
:1031900082E696E062E17AE0F5CF8430A9F782E634
:1031A00096E06EEF79E0EECFCF2DD0E0C930D105BB
:1031B0001CF06F2D685C02C06F2D6F5C82E696E09C
:1031C0000E941F2D82E696E066EF79E00E94FC2CBB
:1031D000BE016F5F7F4F82E696E04AE050E00E94BA
:1031E0008F2E82E696E06BEE79E00E94FC2C8E0139
:1031F0000F5A1B4FD8011196EC91E032F8F482E699
:1032000096E06EED79E00E94FC2CF801818180311E
:1032100030F082E696E063E371E00E94B62ECF5A6A
:10322000DB4F698170E06F7070706F5F7F4F82E677
:1032300096E04AE050E00E94A22E0DC0F0E0EF7050
:10324000F070EE0FFF1FEB54FC4F6081718182E63E
:1032500096E00E94B92EF3948091FD04F81608F4CC
:10326000A3CF82E696E063EC79E00E94FC2C80918B
:1032700069040E94621882E696E068EA79E00E949A
:10328000FC2C80916A040E94621882E696E06DE848
:1032900079E00E94FC2C80916B040E94621882E607
:1032A00096E062E779E00E94FC2C40916104509125
:1032B00062046091630470916404411551056105D5
:1032C000710539F182E696E02AE030E00E94F42DA3
:1032D00082E696E06FE379E00E94FC2C8091650421
:1032E0000E94370AAB01BC0182E696E02AE030E09A
:1032F0000E94F42D82E696E06BE179E00E94FC2CBE
:1033000082E696E0609166044AE050E00E943F2E1B
:1033100006C082E696E062E179E00E943D2D82E6F9
:1033200096E065EF78E00E94FC2C60916704709154
:10333000680482E696E04AE050E00E94192E82E698
:1033400096E068ED78E00E94FC2C609160046031AA
:1033500050F470E06F5F7F4F82E696E04AE050E005
:103360000E94A22E06C082E696E06FEC78E00E94F2
:103370003D2D82E696E062EB78E00E94FC2C809185
:103380005F0480FD03C065E371E002C069E371E0A2
:1033900082E696E00E94B92E82E696E065E978E042
:1033A0000E94FC2C80915F0482700E949C1082E637
:1033B00096E066E778E00E94FC2C80915F048470C0
:1033C0000E949C1082E696E067E578E00E94FC2C63
:1033D00080915F0488700E949C10DF91CF911F91B3
:1033E0000F91FF9008951F93CF93DF9382E696E0AD
:1033F00066E97BE00E94FC2C40912C0450912D0446
:1034000060912E0470912F0482E696E02AE030E06D
:103410000E94F42D82E696E060E87BE00E94FC2C9E
:103420004091300450913104609132047091330422
:1034300082E696E020E130E00E94F42D82E696E0FC
:103440006AE67BE00E94FC2C82E696E06091340400
:103450004AE050E00E943F2E82E696E064E57BE081
:103460000E94FC2C82E696E0609135044AE050E030
:103470000E943F2E82E696E06EE37BE00E94FC2CE9
:10348000C6E3D4E010E012C0112331F082E696E0EA
:103490006DE371E00E94B62E82E696E069914AE003
:1034A00050E00E942D2E1F5F183119F0888188236B
:1034B00059F782E696E00E94272D82E696E068E2C0
:1034C0007BE00E94FC2C82E696E060914E044AE08C
:1034D00050E00E943F2E82E696E063E17BE00E948E
:1034E000FC2CE0914F04F0E0E770F070EE0FFF1F4E
:1034F000EB52FC4F6081718182E696E00E94B92E0A
:1035000082E696E06EEF7AE00E94FC2C80914F04F8
:1035100090E0887190708830910589F0893091052C
:103520001CF4892B39F01BC08031910569F0489754
:10353000B1F40FC082E696E065EF7AE00EC082E655
:1035400096E069EE7AE009C082E696E063EE7AE002
:1035500004C082E696E069ED7AE00E943D2D82E6A5
:1035600096E065EC7AE00E94FC2C40912804509192
:10357000290460912A0470912B0482E696E02AE0E7
:1035800030E00E94F42D82E696E06CEA7AE00E9438
:10359000FC2C80914F0480720E949C1082E696E081
:1035A00063E97AE00E94FC2C80914F0480740E94B1
:1035B0009C1082E696E06AE77AE00E94FC2C8091FB
:1035C0004F0480780E949C1082E696E06DE57AE0D8
:1035D0000E94FC2C87E294E00E94470AAB01BC01E8
:1035E00082E696E02AE030E00E94E52D82E696E051
:1035F00068E57AE00E94FC2C87E294E00E94470A8A
:103600009B01AC0160E472E48FE090E00E94D13550
:1036100082E696E0BA01A9012AE030E00E94E52D99
:1036200082E696E065E57AE00E943D2DDF91CF913C
:103630001F910895EF92FF920F931F937C0102E672
:1036400016E0C8016F2D70E04AE050E00E94082E9D
:10365000C8016EE20E941F2DB70154E07695679570
:103660005A95E1F76F707070C8014AE050E00E940F
:10367000082EC8016EE20E941F2D8FE0E822FF2471
:10368000C801B7014AE050E00E94082E1F910F9137
:10369000FF90EF9008950F931F93CF93DF932091A6
:1036A00074042F3FA9F582E696E067ED75E00E946D
:1036B000FC2C86E593E00E941A1B82E696E066EBFE
:1036C00075E00E94FC2C8091FE049091FF040E9402
:1036D0001A1B82E696E063E875E00E943D2D82E6C3
:1036E00096E060E675E00E943D2D82E696E068E493
:1036F00075E00E943D2D82E696E063E275E00E944F
:103700003D2D82E696E00E94272D0E94AF1869C0E9
:1037100012160CF066C0332727FD30958091FD040A
:1037200090E0821793070CF45CC082E696E06EE0AE
:1037300075E00E94FC2C60917404772767FD7095FA
:1037400082E696E04AE050E00E94A22E82E696E0F1
:1037500063EE74E00E94FC2C10E008E23AC0C12F36
:10376000D0E0CC0FDD1FC452DB4F288130E08091C8
:103770007404992787FD909501972817390741F51B
:1037800082E696E06FE371E00E94B62E82E696E054
:10379000602F4AE050E00E942D2E82E696E063E41E
:1037A00071E00E94B62EE981F0E0EF70F070EE0F4C
:1037B000FF1FEB54FC4F6081718182E696E00E940E
:1037C000B62E82E696E067E471E00E94B62E0F5FA7
:1037D0001F5F8091FC04181710F282E696E00E94A9
:1037E000272DDF91CF911F910F910895CF92DF92F6
:1037F000EF92FF920F931F93DF93CF93CDB7DEB776
:103800006C970FB6F894DEBF0FBECDBF282F809106
:1038100074048F3F09F050C1822F992787FD90953E
:10382000A92FB92FFC013A97EF36F10508F03DC1F9
:10383000EA5AFF4FEE0FFF1F0590F491E02D099417
:1038400082E696E069E471E0B4C082E696E069E45D
:1038500071E00E94B92E22C182E696E065E571E032
:103860000E94B92E85E78983DE011296E1E5F4E036
:103870008BE101900D928150E1F7CE0101966CE150
:103880000E9429110E94CB0D83E08093260468ECEE
:1038900070E080E090E00E94502A809126048430FD
:1038A00009F003C18FE70E94E00B0E94F40B8983AB
:1038B000853509F0FAC082E696E065EC74E00E9476
:1038C0003D2D82E696E067EA74E00E943D2D82E697
:1038D00096E069E874E0B2C082E696E06DE671E0D9
:1038E0000E94B92E89E68983CE01019661E00E948B
:1038F00029110E94CB0D83E08093260468EC70E0D0
:1039000080E090E00E94502A80912604843009F0E3
:10391000CCC08FE70E94E00B0E94F40B89838E01DC
:103920000E5F1F4FBDE1EB2EF12CEC0EFD1E0E9431
:10393000F40BD8018D938D01AE15BF05C1F7A1E53C
:10394000B4E0FE0132968BE101900D928150E1F7D7
:103950008981893409F0A9C082E696E06BE674E0BB
:103960000E943D2D82E696E06DE474E00E943D2DBC
:1039700082E696E06FE274E061C082E696E067E876
:1039800071E00E94B92E8EEF809374048EC0205295
:103990002750422F4053242F332727FD3095809105
:1039A000FD0490E0821793073CF482E696E066E916
:1039B00071E00E94B92E79C0409374046FC084E115
:1039C0008093740482E696E068EF73E037C085E187
:1039D0008093740482E696E061EC73E02FC086E188
:1039E0008093740482E696E06AE873E027C087E17A
:1039F0008093740482E696E060E473E01FC088E17F
:103A00008093740482E696E06FE273E017C089E168
:103A10008093740482E696E06BE173E00FC08AE164
:103A20008093740482E696E066E073E007C08BE161
:103A30008093740482E696E06EED72E00E943D2D64
:103A400034C082E696E064EC72E00E943D2D8091E5
:103A50005F0491E01DC082E696E06EEA72E00E948B
:103A60003D2D80915F0492E013C082E696E069E903
:103A700072E00E943D2D80915F0494E009C082E6CF
:103A800096E06EE772E00E943D2D80915F0498E021
:103A9000892780935F048FEF809374040E944B1BEF
:103AA00004C082E696E00E94E42B82E696E00E9443
:103AB000BD2B892BB1F776C1822F0E94B0178823C6
:103AC00009F470C18091DA04882321F48FEF809388
:103AD000740460C185E794E060E070E040E050E08D
:103AE0000E9481079B01AC0190917404963109F406
:103AF0007CC0973164F4943109F463C095310CF0C3
:103B00006AC0892F81508D3008F034C113C09931BB
:103B100009F4E5C09A313CF4973109F470C098314A
:103B200009F028C1D2C09A3109F4E7C09B3109F0ED
:103B300021C1F4C0E92FFF27E7FDF0958091FD0436
:103B400090E08E179F070CF415C1DA01C9010197A7
:103B5000A109B1098097A105B10548F0A8E2FA2EA4
:103B600000E010E06F010894C108D10825C0EF5AA9
:103B7000FB4F822F81508083E5C0612F70E0660F7C
:103B8000771F64527B4FFB01808190E08C159D056F
:103B900091F48F2D90E0A0E0B0E082179307A40786
:103BA000B50741F4F601EF5AFB4FDB0111968C91FA
:103BB000818301E0F3941F5F8091FC041817E8F201
:103BC000BFC02F3F31054105510511F008F0D2C0AB
:103BD00020936904B7C02F3F31054105510511F00D
:103BE00008F0C8C020936A04ADC02F3F31054105DD
:103BF000510511F008F0BEC020936B04A3C0809162
:103C000075048062803719F586E794E060E070E023
:103C100040E050E00E9481079B01AC01DC01CB0138
:103C20000197A109B1090897A105B10508F0B5C030
:103C3000CA01B90124ED30E340E050E00E949F3515
:103C40009B01AC012A5E3C4A4A46554E24C086364A
:103C500011F586E794E060E070E040E050E00E94FB
:103C600081079B01AC01DC01CB010197A109B109DE
:103C70000797A105B10508F090C0CA01B90128EA6B
:103C800031E640E050E00E949F359B01AC01245E8C
:103C90003C434E46544E211531054105510561F016
:103CA000DA01C9018054914EAD49B8418158904F15
:103CB000AA4FB24008F05EC02093610430936204C2
:103CC00040936304509364043DC02F3F3105410588
:103CD000510511F008F04EC02093650433C0DA019D
:103CE000C9010197A109B1098F3F9105A105B1054E
:103CF00008F040C02093660425C0DA01C901845C45
:103D00009940A040B0408D549D41A040B04030F457
:103D1000309368042093670401E001C000E021159E
:103D200031054105510511F48FEF07C021313105EF
:103D30004105510528F4822F81508093600402C010
:103D40000023C1F08091DB048823D1F480913004FA
:103D500090913104A0913204B09133040196A11DD9
:103D6000B11D8093300490933104A0933204B0933A
:103D7000330406C082E696E068EA71E00E94B92E3C
:103D80000E94A6178FEF8093740482E696E06AE0A3
:103D90000E94512D0E944B1B05C021E030E040E005
:103DA00050E07ECF6C960FB6F894DEBF0FBECDBF4D
:103DB000CF91DF911F910F91FF90EF90DF90CF9007
:103DC000089582E696E062E372E00E943D2D82E66D
:103DD00096E06AE172E00E943D2D82E696E00E9444
:103DE000BD2B892B31F082E696E00E94E42B0E94E5
:103DF000F61B0E94F512823019F0833069F405C079
:103E000082E696E06CEF71E004C082E696E065EE33
:103E100071E00E943D2D08958FEF809374041092FD
:103E2000DB040E944B1B0CC082E696E00E94BD2B77
:103E3000892B31F082E696E00E94E42B0E94F61B6B
:103E4000809174048E3F81F70895809174048430CA
:103E500009F46FC0853084F4813009F45BC082308E
:103E600024F48F3F09F085C014C0823009F457C094
:103E7000833009F07EC058C0863009F464C08630B3
:103E80000CF45CC0873009F463C0893009F071C05C
:103E90006AC082E696E06AE478E00E943D2D86E5FD
:103EA00093E00E941A1B82E696E062E378E00E94AB
:103EB0003D2D82E696E06DE078E00E943D2D82E6A1
:103EC00096E063EE77E00E943D2D82E696E062EC9C
:103ED00077E00E943D2D82E696E065E977E00E945A
:103EE0003D2D82E696E06FE677E00E943D2D82E66A
:103EF00096E06BE477E00E943D2D82E696E064E276
:103F000077E00E943D2D82E696E00E94272D0E94D8
:103F1000F3192FC082E696E067E077E028C082E6DA
:103F200096E062EE76E023C082E696E06DEC76E005
:103F30001EC082E696E06EEA76E019C082E696E060
:103F40006AE676E014C082E696E065E576E00FC0AA
:103F500082E696E060E476E00E943D2D82E696E0FF
:103F60006AEF75E004C082E696E064EE75E00E94B8
:103F70003D2D6AE070E080E090E00E94502A04C08D
:103F800082E696E00E94E42B82E696E00E94BD2B3A
:103F9000892BB1F708952F923F924F925F926F92C3
:103FA0007F928F929F92AF92BF92CF92DF92EF92C9
:103FB000FF920F93DF93CF93CDB7DEB7A8970FB6DD
:103FC000F894DEBF0FBECDBF7E010894E11CF11C4A
:103FD00080E1D7011D928A95E9F782E696E066ECCA
:103FE00071E00E94B92E0E94BA1320E431EE4DE92F
:103FF00058E129A33AA34BA35CA380EC91EDA8E977
:10400000BBE18D8F9E8FAF8FB8A324EF31E040E0EE
:1040100050E0298F3A8F4B8F5C8F20E5822E23EC66
:10402000922EA12CB12C80E491EEADE9B8E18D8BFC
:104030009E8BAF8BB88F44245524320100E022249C
:104040003324198A1A8A1B8A1C8A0DC182E696E0DB
:104050000E94E42B8434C9F0853434F48332C9F1EE
:104060008C3209F0CEC046C0833509F0CAC029A100
:104070003AA14BA15CA1C901DA018D8B9E8BAF8B5C
:10408000B88F442455243201EEC082E696E064E401
:104090000E941F2D82E696E040E451EE6DE978E142
:1040A0002AE030E00E94532E82E696E06CE20E9405
:1040B0001F2D82E696E040EC51ED68E97BE12AE0B5
:1040C00030E00E94532E82E696E06CE20E94512D71
:1040D000CAC019821A821B821C821D821E821F8204
:1040E000188619861A861B861C861D861E861F86C4
:1040F000188A3CC00F5F043009F0B5C069817A812D
:104100008B819C8128EE33E040E050E00E949F3597
:1041100069A37AA38BA39CA36D817E818F819885EF
:104120000E949F356D8F7E8F8F8F98A329853A854A
:104130004B855C85298F3A8F4B8F5C8F6D857E8593
:104140008F85988928EE33E040E050E00E949F354B
:104150004B015C0160323EE4730730E0830730E0DE
:10416000930730F48CE162E30E940A0C00E07BC00C
:10417000603345E7740740E0840740E0940718F493
:104180008CE162E2F1CF60345CE9750750E08507AD
:1041900050E0950718F48CE166E2E6CF80E58816DA
:1041A00083EC980680E0A80680E0B80618F48CE15D
:1041B00062E1DACF90E689169AEE990690E0A906B8
:1041C00090E0B90618F48CE165E1CECFA0E78A163D
:1041D000A1E19A06A1E0AA06A0E0BA0618F48CE1D3
:1041E00061E0C2CFB0EA8B16B6E89B06B1E0AB0641
:1041F000B0E0BB0618F48CE163E0B6CF8CE165E07B
:10420000B3CF80538A3078F5C02EDD24CC0CDD1C72
:10421000CC0CDD1CE1E0F0E0EC0FFD1FCE0EDF1E4C
:10422000282F332727FD3095432F532F2DA33EA34F
:104230004FA358A7D6016D917D918D919C912AE055
:1042400030E040E050E00E949F352DA13EA14FA1FB
:1042500058A5260F371F481F591FD6012D933D9390
:104260004D935C93139782E696E00E94BD2B892BB9
:1042700009F0ECCE411451046104710499F46D8984
:104280007E898F89988D0E94800C61E070E080E0CB
:1042900090E00E94502A22242A943324198A1A8AF0
:1042A0001B8A1C8A298D3A8D4B8D5C8D42165306D4
:1042B00064067506D0F40E942B0C29893A894B8933
:1042C0005C89280F311D411D511D298B3A8B4B8B69
:1042D0005C8B381608F4382E821508F4282E0894C2
:1042E000411C511C611C711C64C06D897E898F89C1
:1042F000988D28EE33E040E050E00E94D13582E610
:1043000096E0BA01A9012AE030E00E94E52D82E69C
:1043100096E06CE20E941F2D82E696E0632D4AE053
:1043200050E00E942D2E82E696E06CE20E941F2D46
:1043300069897A898B899C89A30192010E94D13570
:1043400082E696E0BA01A9012AE030E00E94E52D5C
:1043500082E696E06CE20E941F2D82E696E0622DD6
:104360004AE050E00E942D2E82E696E06CE20E9428
:10437000512D8D899E89AF89B88D880D991DAA1DF3
:10438000BB1D8D8B9E8BAF8BB88F2D8D3E8D4F8D32
:1043900058A1281739074A075B0740F489A19AA159
:1043A000ABA1BCA18D8B9E8BAF8BB88F44245524C1
:1043B000320129A13AA14BA15CA1285E33404040C3
:1043C000504009F050CFA8960FB6F894DEBF0FBE4C
:1043D000CDBFCF91DF910F91FF90EF90DF90CF9005
:1043E000BF90AF909F908F907F906F905F904F9015
:1043F0003F902F900895EF92FF920F931F93DF93BA
:10440000CF93CDB7DEB7CA55D0400FB6F894DEBF14
:104410000FBECDBF8B017A01893009F4ADC08A305F
:10442000E0F4843009F465C0853050F4823009F43A
:1044300047C0833008F055C0813009F0D4C12FC087
:10444000863009F47FC0863008F460C0873009F4F4
:1044500083C0883009F0C7C187C0893609F427C1F5
:104460008A3680F4863609F4D4C0873620F485363F
:1044700009F0B9C1B5C0873609F4E4C0883609F03F
:10448000B2C1E6C08B3609F45AC18B3608F417C1A5
:104490008C3609F466C1873C09F0A5C197C181E05B
:1044A00069E270E00E94871707E214E0F801819149
:1044B0008F010E947017F4E000351F07B9F79BC108
:1044C00082E06BE170E00E94871701E514E0F801DB
:1044D00081918F010E947017F4E00C361F07B9F725
:1044E0008AC183E061E070E00E9487170E94F512A4
:1044F00080C184E061E070E00E94871781E00E9443
:1045000070170E9469170E94CB1F77C16091FC044D
:1045100070E0660F771F85E00E94871700E010E0CB
:1045200008C0F801E452FB4F80810E9470170F5FB2
:104530001F4F8091FC0490E0880F991F08171907FE
:1045400080F359C186E062E070E00E94871786E53B
:1045500093E00E947E174FC187E061E070E00E9407
:1045600087178091FD0445C188E061E070E00E94FA
:104570008717809150043DC186E68983CE0101965C
:1045800061E00E9429110E94CB0D83E080932604F4
:1045900068EC70E080E090E00E94502A8091260450
:1045A0008430E1F48FE70E94E00B0E94F40B8983D2
:1045B000863471F489E060E270E00E94871710E0B1
:1045C0000E94F40B0E9470171F5F1032C9F713C1CD
:1045D00089E061E070E00E948717F6C089E004C1BD
:1045E00085E661E070E00E9487170932110509F045
:1045F000FFC020E030E0F901E95DFB4FD701A20FD9
:10460000B31F8C9180832F5F3F4F2932310599F77B
:10461000DBC086E661E070E00E9487170B31110570
:1046200009F0E6C020E030E0F901EF5AFB4FD70176
:10463000A20FB31F8C9180832F5F3F4F2B31310529
:1046400099F7C2C087E661E070E00E94871786C0D4
:1046500088E661E070E00E94871785E78A83DE01C3
:104660001396E1E5F4E08BE101900D928150E1F7C2
:10467000CE0102966CE10E9429110E94CB0D83E0CD
:104680008093260468EC70E080E090E00E94502A5D
:1046900080912604843009F0ABC08FE70E94E00BC4
:1046A0000E94F40B8A83853509F0A2C08DC089E68B
:1046B00061E070E00E9487170E94BF0985C08AE60A
:1046C00061E070E00E94871789E68E8FCE014E96DA
:1046D00061E00E9429110E94CB0D83E080932604A3
:1046E00068EC70E080E090E00E94502A80912604FF
:1046F000843009F07DC08FE70E94E00B0E94F40B2C
:104700008E8F8E01015E1F4F3AE3E32EF12CEC0EEB
:10471000FD1E0E94F40BF80181938F01EE15FF0539
:10472000C1F7A1E5B4E0FE017F968BE101900D9207
:104730008150E1F78E8D893409F05AC045C08BE66F
:1047400061E070E00E948717F70180810E947C146D
:104750000E946F09892BC1F50E94BF090E941114A4
:1047600033C08CE661E070E00E94871700321105CB
:1047700071F487E68AAFDE01DB96F70180E20190F3
:104780000D928150E1F7CE01CA9661E205C087E43F
:104790008AAFCE01CA9661E00E9429110E94CB0D1A
:1047A00083E08093260468EC70E080E090E00E9453
:1047B000502A809126048430D9F48FE70E94E00BC0
:1047C0000E94F40B8734A1F481E013C087EC61E010
:1047D00070E00E94871781E00E9470170E9469179D
:1047E000109272040AC08AEC61E070E00E948717A0
:1047F00080E00E9470170E946917C65ADF4F0FB6FB
:10480000F894DEBF0FBECDBFCF91DF911F910F9106
:10481000FF90EF900895AF92BF92CF92DF92EF9208
:10482000FF920F931F93CF93DF93B4E0AB2EA6E0DC
:10483000BA2EF5E0CF2E08EA15E0E4E6DE2E72E0AF
:10484000E72E63E0F62EA1C082E696E00E94E42BFC
:10485000982F8093130680911206833021F18430C3
:1048600028F4813099F08230B8F409C0853009F419
:1048700048C0853020F1863009F087C05FC0953B85
:1048800009F083C081E0809312067FC0923609F060
:104890007AC0E092120679C09093110690931006A8
:1048A000F092120672C090930E0610920F0680913D
:1048B0001006892780931006A092120666C0D92F91
:1048C000C0E020910E0630910F062C2B3D2B30932B
:1048D0000F0620930E0680911006892780931006FC
:1048E000C09212062536310508F44FC08CEC61E009
:1048F00070E00E94871781E00E9470170E9469177C
:1049000042C020910C0630910D06F901E855FA4F8E
:104910009083809110068927809310062F5F3F4F68
:1049200030930D0620930C0680910E0690910F0691
:104930002817390750F1B092120627C0809110064F
:10494000891759F460910C0670910D06809111063B
:1049500048EA55E00E94FB210DC08BEC62E070E05C
:104960000E948717809111060E947017809173042E
:104970000E947017F8018D2D11928A95E9F7109217
:104980000D0610920C061092120682E696E00E9426
:10499000BD2B892B09F058CFDF91CF911F910F913B
:1049A000FF90EF90DF90CF90BF90AF90089581E09F
:1049B0008093720408C082E696E00E94BD2B892B8A
:1049C00011F00E940B24809172048823A1F70895AE
:1049D000DF92EF92FF920F931F93CF93DF930E948A
:1049E0002A2A6115710581059105C9F30E9478078E
:1049F0001092300410923104109232041092330459
:104A0000DD24E0903004F0903104009132041091E4
:104A10003304102F0F2DFE2CEE240E9473072FEF6E
:104A200030E040E050E00E94F335E60EF71E081F2C
:104A3000191FE0923004F092310400933204109375
:104A40003304D39484E0D816E1F6C6E3D4E010E052
:104A500017C00E94730722E330E040E050E00E945C
:104A6000F3356F5FE6E3F4E090E004C081918617D0
:104A700081F39F5F9117D0F369931F5F183119F08D
:104A80008881882331F7DF91CF911F910F91FF909B
:104A9000EF90DF9008951F93109174041F3F09F069
:104AA000BFC0893409F466C08A342CF5883309F410
:104AB00076C089336CF4803309F481C081330CF003
:104AC0006CC08B3109F44CC0813209F0A3C03CC0EA
:104AD000813409F483C082343CF4893309F46DC015
:104AE000803409F097C030C0823409F482C0863423
:104AF00009F090C04FC0823609F47BC083368CF435
:104B0000883571F1893534F48235E9F1833509F05E
:104B100081C01FC08A3509F478C0813609F07AC097
:104B20005DC0823781F1833734F4863699F1893656
:104B300009F070C01FC0883799F08A3709F465C042
:104B4000833709F067C005C082E696E069E471E04A
:104B500017C00E94111482E696E063ED71E006C072
:104B60000E946F0982E696E06DEE71E00E94B92E18
:104B70008EEF4EC00E94BF0982E696E06CE072E0C4
:104B80000E94B92E47C00E94E82482E696E065E2C2
:104B900072E0F6CF0E9419183DC0805339C082E6FA
:104BA00096E062ED71E00E943D2D90914F04892FB7
:104BB000885F8871977E892B0CC089E029C082E6C6
:104BC00096E06FEB71E00E943D2D80914F0490E2E2
:104BD000892780934F04109374041CC082E696E0EA
:104BE00069EA71E00E943D2D80914F0490E489278D
:104BF00009C082E696E068E971E00E943D2D80914F
:104C00004F04805880934F0402C00E94E11E8FEF32
:104C100080937404809174048E3F09F4E8C0DFC06F
:104C20000E94B017882309F4E2C08091DA04882337
:104C300021F48FEF80937404D2C085E794E060E0A4
:104C400070E040E050E00E9481079B01AC01809140
:104C50007404843009F441C0853044F4823041F159
:104C6000833094F5813009F096C00DC0863009F488
:104C700067C086300CF43EC0873009F469C08930C3
:104C800009F089C075C0DA01C9018154914EAD495E
:104C9000B8418F57904FAA4FB24008F07CC0209384
:104CA0002C0430932D0440932E0450932F049AC06B
:104CB00020933004309331044093320450933304F2
:104CC00081E08093DB048EC0283031054105510519
:104CD00008F061C02093340485C0DA01C90101974E
:104CE000A109B1090A97A105B10508F054C02093A4
:104CF000350478C085E794E06DE371E00E949D087B
:104D000010E00EC0183130F4E12FF0E0E95DFB4F08
:104D100087871F5F80E090E06DE371E00E949D084F
:104D2000009759F00E947F08009761F706C0E12FB5
:104D3000F0E0E95DFB4F17861F5F1831C0F352C0EA
:104D4000253031054105510530F520934E044AC008
:104D5000DA01C9010197A109B1090697A105B105B9
:104D6000D0F480914F04887F822B80934F043AC007
:104D7000DA01C9010197A109B1098050924CA14003
:104D8000B04048F4209328043093290440932A0427
:104D900050932B0427C082E696E068EA71E00E94F7
:104DA000B92E13C08091300490913104A091320447
:104DB000B09133040196A11DB11D809330049093EE
:104DC0003104A0933204B09333040E94A6178FEFEE
:104DD0008093740482E696E06AE00E94512D0E945E
:104DE000251F05C08091DB048823E1F2EECF1F91DF
:104DF00008958FEF809374041092DB040E94251FA6
:104E00000CC082E696E00E94BD2B892B31F082E631
:104E100096E00E94E42B0E944B25809174048E3F03
:104E200081F76AE070E080E090E00E94502A04C0C0
:104E300082E696E00E94E42B82E696E00E94BD2B7B
:104E4000892BB1F708957F928F929F92AF92BF9274
:104E5000CF92DF92EF92FF920F931F93DF93CF9346
:104E6000CDB7DEB7AA970FB6F894DEBF0FBECDBFA1
:104E70000E941C2A7B018C0181E00E94EC0C04C082
:104E800082E696E00E94E42B82E696E00E94BD2B2B
:104E9000892BB1F75F98DD24D39432E6732E22E09C
:104EA000822E912C8C0E9D1E5E010894A11CB11CBB
:104EB00093E0C92E0E941C2A20E030E06E197F0981
:104EC000800B910B693C71058105910510F021E083
:104ED00030E08D2D90E028233923232B99F10E9477
:104EE0001C2A7B018C01469A80ED97E00E94EB081A
:104EF0007982D401E7E2F4E089E201900D928150D9
:104F0000E1F7C5016AE20E942911469880E090E02D
:104F10000E94EB08C09226040E94CB0D62E370E071
:104F200080E090E00E94502A80912604843051F461
:104F3000C09226048FE70E94E00B0E94F40B82349B
:104F400009F4DD2482E10E948C2B892B49F5DD24B4
:104F5000D39426C05F9A469A82E696E00E94E42B9C
:104F60008D30910569F08E3091051CF40A97B1F4EB
:104F700007C08332910569F08234910579F40CC041
:104F800082E696E06AE871E00E943D2D0E94F926D3
:104F900005C00E94CB1F02C00E94D7245F9846988C
:104FA00082E696E00E94BD2B892B09F483CFD2CFF5
:104FB00082E696E00E94BD2B04970CF182E696E013
:104FC0000E94E42B82349105D1F482E696E00E949F
:104FD000E42B8E34910599F482E696E00E94E42B4E
:104FE0008434910561F482E696E00E94E42B819777
:104FF00031F480E090E00E94EB080E94232708959E
:105000008F929F92AF92BF92CF92DF92EF92FF92D8
:105010000F931F9382E10E948C2B892B09F0ACC067
:1050200068EC70E080E090E00E94502A80E090E020
:105030000E94EB080E941C2A5B016C0140ECE42EEC
:1050400042E1F42E012D112DE60EF71E081F191F47
:1050500006C082E10E948C2B892B09F085C00E943A
:105060001C2A6E157F058007910798F382E10E9444
:105070008C2B892B09F078C080ED97E00E94EB081B
:105080000E941C2A7B018C0199249394882488E433
:1050900096E2A0E0B0E0A80EB91ECA1EDB1E29C031
:1050A000AE14BF04C006D10638F480ED97E00E942C
:1050B000EB08882483941DC00E941C2A6E197F0966
:1050C000800B910B693C71058105910590F00E9460
:1050D0001C2A7B018C0180E0992009F481E0982E44
:1050E000882319F480E090E002C080ED97E00E94F0
:1050F000EB0882E10E948C2B892B91F280E090E0FA
:105100000E94EB08882051F1809150048F5F8370DA
:105110000E947C1482E696E062E472E00E94B62E61
:1051200082E696E0609150044AE050E00E943F2EF3
:105130000E946F09892B39F082E696E06FE472E0F5
:105140000E94B92E19C082E696E06CE672E00E94D9
:10515000B62E0E94BF090E9411140EC00E94E824BE
:105160000E9411140E94F31982E696E06EE872E044
:105170000E94B92E0E9423271F910F91FF90EF905C
:10518000DF90CF90BF90AF909F908F900895EF9257
:10519000FF920F931F9380E00E944A090E94DD1244
:1051A00086E061E00E94CC2A85E061E00E94CC2A82
:1051B00082E160E00E94CC2A84E060E00E94CC2A78
:1051C00084E061E00E94592B0E94E91282E696E099
:1051D00060E072EC0E94BC2B0E946B140E946F096D
:1051E000892B39F082E696E06FE472E00E94B92ED6
:1051F0000AC082E696E06CE672E00E94B62E0E943B
:10520000BF090E9411140E94900E8FEF8093310508
:105210000E94170978940E941C2A7B018C018091BE
:1052200031058F3F09F0B6C00E941C2A6E197F0914
:10523000800B910B605D77408040904008F0AAC0E1
:10524000EECF82E696E00E94E42B82E696E00E9492
:10525000BD2B892BB1F782E696E065EA72E00E94E9
:10526000B62E86E593E00E941A1B82E696E06CEB70
:1052700072E00E94B62E82E696E066E070E04AE0B8
:1052800050E00E94A22E68EC70E080E090E00E9466
:10529000502A0E94D82740912804509129046091F7
:1052A0002A0470912B04DB01CA010197A109B109FD
:1052B0000497A105B10568F440933205433029F005
:1052C00040E052EC61E070E004C040EA56E861E082
:1052D00070E088EF96E00E94882F0E9400285F9877
:1052E00080E090E00E94EB080E94900E80E00E9417
:1052F000EC0C809117050E94150C0E94CB0D1092AA
:105300009C0510929D0510929E056CE271E080E074
:1053100090E00E94502A80ED97E00E94EB0864E63E
:1053200070E080E090E00E94502A80E090E00E94CF
:10533000EB0810E015C064E670E080E090E00E94A9
:10534000502A80ED97E00E94EB0864E670E080E070
:1053500090E00E94502A80E090E00E94EB081F5FDE
:1053600080915004181738F380914F0490E084FF27
:1053700009C020E088719070489709F421E0822FDD
:105380000E948C148FE00E944A091F910F91FF9098
:10539000EF90089580ED97E00E94EB0882E161E0D4
:1053A0000E94592B5F9A51CF1F920F920FB60F9206
:1053B00011242F933F938F939F93AF93BF9380912B
:1053C000190690911A06A0911B06B0911C06309107
:1053D0001D060196A11DB11D232F2D5F2D3720F035
:1053E0002D570196A11DB11D20931D06809319060E
:1053F00090931A06A0931B06B0931C068091150685
:1054000090911606A0911706B09118060196A11D5D
:10541000B11D8093150690931606A0931706B093BE
:105420001806BF91AF919F918F913F912F910F904F
:105430000FBE0F901F9018958FB7F8942091190602
:1054400030911A0640911B0650911C068FBFB9017E
:10545000CA0108959FB7F894209115063091160659
:10546000409117065091180686B5A89B06C08F3F3D
:1054700021F02F5F3F4F4F4F5F4F9FBF542F432F60
:10548000322F2227280F311D411D511D82E0220F8E
:10549000331F441F551F8A95D1F7B901CA010895DA
:1054A000EF92FF920F931F93CF93DF937B018C01B9
:1054B0000E942A2AEB010EC00E942A2A6C1B7D0B37
:1054C000685E7340C8F30894E108F1080109110906
:1054D000C851DC4FE114F1040105110569F7DF91B2
:1054E000CF911F910F91FF90EF900895789484B51C
:1054F000826084BD84B5816084BD85B5826085BDD0
:1055000085B5816085BDEEE6F0E0808181608083B5
:10551000E1E8F0E010828081826080838081816098
:105520008083E0E8F0E0808181608083E1E9F0E061
:10553000808182608083808181608083E0E9F0E007
:10554000808181608083E1ECF0E0808184608083F1
:10555000808182608083808181608083E3ECF0E0E1
:10556000808181608083E0ECF0E0808182608083D4
:10557000E2ECF0E0808181608083EAE7F0E0808106
:105580008460808380818260808380818160808369
:105590008081806880830895CF93DF93482F50E007
:1055A000CA018C50944FFC0134914A52544FFA0175
:1055B0008491882369F190E0880F991FFC01E455DC
:1055C000F44FA591B491FC01E654F44FC591D491E8
:1055D000662351F42FB7F8948C91932F90958923DB
:1055E0008C93888189230BC0623061F42FB7F894C3
:1055F0008C91932F909589238C938881832B88831A
:105600002FBF06C09FB7F8948C91832B8C939FBFBC
:10561000DF91CF910895883071F1893068F482303C
:1056200031F1833020F4813009F042C01DC0833055
:1056300089F08430E9F512C08B3059F18C3028F4B0
:105640008930E9F08A30A1F51EC08C3031F18E30FE
:1056500079F529C0809180008F7703C08091800008
:105660008F7D80938000089584B58F7702C084B5C4
:105670008F7D84BD0895809190008F7707C08091C1
:1056800090008F7D03C080919000877F8093900071
:1056900008958091C0008F7703C08091C0008F7DF6
:1056A0008093C00008958091C200877F8093C200DC
:1056B0000895FF920F931F93F62E482F50E0CA01D2
:1056C0008E5E934FFC012491CA018C50944FFC01D3
:1056D00014914A52544FFA0104910023C9F0222335
:1056E00019F0822F0E940B2BE02FF0E0EE0FFF1F2E
:1056F000E654F44FA591B4919FB7F894FF2021F49C
:105700008C911095812302C08C91812B8C939FBF2B
:105710001F910F91FF9008950F931F93482F50E012
:10572000CA018E5E934FFC012491CA018C50944FA4
:10573000FC0104914A52544FFA011491112319F4B7
:1057400020E030E015C0222319F0822F0E940B2B9D
:10575000812F90E0880F991F8853944FFC01A591E9
:10576000B4918C9120E030E0802311F021E030E012
:10577000C9011F910F910895089520915E063091FF
:105780005F068091600690916106281B390B2F738C
:105790003070C901089520915E0630915F068091B6
:1057A0006006909161062817390719F42FEF3FEF33
:1057B00009C0E0916006F0916106E25EF94F8081D8
:1057C000282F30E0C901089520915E0630915F06D0
:1057D00080916006909161062817390719F42FEF20
:1057E0003FEF13C0E0916006F0916106E25EF94F71
:1057F0002081809160069091610601968F73907070
:10580000909361068093600630E0C901089510927C
:1058100065061092640688EE93E0A0E0B0E0809305
:10582000660690936706A0936806B093690687EFB3
:1058300093E0909363068093620608950F931F93FD
:10584000DF93CF930F92CDB7DEB78C016983809140
:10585000B203882369F083E0BE016F5F7F4F41E0B0
:1058600050E00E941C321816190614F49C0107C05F
:1058700081E090E0F8019383828320E030E0C90169
:105880000F90CF91DF911F910F91089583E00E94B7
:10589000F3310895CF93DF9312C082E00E94643108
:1058A0002FEF8F3F9207C9F0E0915E06F0915F06FF
:1058B000E25EF94F8083D0935F06C0935E06C0918D
:1058C0005E06D0915F062196CF73D07080916006FE
:1058D00090916106C817D90701F7DF91CF9108951C
:1058E000FC0180818E5F808380E86CE37CE042E491
:1058F00050E00E949A310895FC0181819081913A93
:1059000059F4813209F04CC080E06BEA73E047E063
:1059100050E00E949A3142C0913209F041C0803279
:1059200039F48BEA93E067E070E00E94DE3136C024
:10593000823209F035C082818093B2038091AB033B
:105940009091AC03A091AD03B091AE03805B944005
:10595000A040B04019F58091B20380FD12C087E7E6
:1059600097E790930108809300082BE088E190E08E
:105970000FB6F894A895809360000FBE2093600046
:105980000DC088E10FB6F89480936000109260001B
:105990000FBEA895109201081092000881E00895AA
:1059A00080E00895CF92DF92EF92FF920F931F93C2
:1059B000CF93DF937C016B018A01C0E0D0E00FC080
:1059C000D6016D916D01D701ED91FC910190F081AF
:1059D000E02DC7010995C80FD91F015010400115CE
:1059E000110571F7CE01DF91CF911F910F91FF90BB
:1059F000EF90DF90CF900895EF92FF920F931F9357
:105A0000CF93DF937C018B01C0E0D0E0F8010F5F02
:105A10001F4F6491662359F0D701ED91FC910190DD
:105A2000F081E02DC7010995C80FD91FEFCFCE0136
:105A3000DF91CF911F910F91FF90EF900895DC01BE
:105A4000ED91FC910190F081E02D09950895EF9280
:105A5000FF920F931F938C016DE00E941F2D7C011C
:105A6000C8016AE00E941F2D9C012E0D3F1DC90137
:105A70001F910F91FF90EF900895EF92FF920F9377
:105A80001F937C010E94FC2C8C01C7010E94272DD2
:105A90009C01200F311FC9011F910F91FF90EF90C2
:105AA0000895EF92FF920F931F937C010E941F2D88
:105AB0008C01C7010E94272D9C01200F311FC901B5
:105AC0001F910F91FF90EF900895CF93DF93EC011A
:105AD0006115710519F420E030E00FC0DB010D9075
:105AE0000020E9F71197A61BB70BE881F981028026
:105AF000F381E02DAD0109959C01C901DF91CF91A2
:105B000008954F925F927F928F929F92AF92BF9231
:105B1000CF92DF92EF92FF920F931F93DF93CF9379
:105B2000CDB7DEB7A1970FB6F894DEBF0FBECDBFDD
:105B30002C01742ECB01223008F42AE019A231E2A4
:105B4000C32ED12CCC0EDD1E822E9924AA24BB2478
:105B5000672D752FA50194010E94D13579018A0125
:105B6000C801B701A50194010E949F35472D461B2E
:105B70000894C108D1084A3014F4405D01C0495C62
:105B8000F6014083E114F1040105110521F07E2C9A
:105B90005F2DC801DDCFC201B6010E94652DA1961F
:105BA0000FB6F894DEBF0FBECDBFCF91DF911F912E
:105BB0000F91FF90EF90DF90CF90BF90AF909F90AC
:105BC0008F907F905F904F900895DC0121153105F3
:105BD00041F4ED91FC910190F081E02D642F099545
:105BE00008950E94812D0895EF92FF920F931F93C5
:105BF0007C010E94E52D8C01C7010E94272D9C018C
:105C0000200F311FC9011F910F91FF90EF90089550
:105C1000EF92FF920F931F939A017B0100E010E037
:105C2000B801A7010E94E52D1F910F91FF90EF9001
:105C30000895EF92FF920F931F937C010E94082E0C
:105C40008C01C7010E94272D9C01200F311FC90123
:105C50001F910F91FF90EF900895EF92FF920F9395
:105C60001F939A01E62EFF2400E010E0B801A7017F
:105C70000E94E52D1F910F91FF90EF900895EF92F4
:105C8000FF920F931F937C010E942D2E8C01C70160
:105C90000E94272D9C01200F311FC9011F910F91D8
:105CA000FF90EF900895CF92DF92EF92FF920F93C3
:105CB0001F93CF93DF93EC016A017B01211531051E
:105CC00041F4E881F9810190F081E02D642F09957C
:105CD0001BC02A303105B1F477FF13C06DE20E947A
:105CE0001F2D8C0144275527BA014C195D096E09F7
:105CF0007F09CE012AE00E94812D9C01200F311FD7
:105D000004C02AE00E94812D9C01C901DF91CF913E
:105D10001F910F91FF90EF90DF90CF900895EF9239
:105D2000FF920F931F937B019A010027F7FC0095C8
:105D3000102FB801A7010E94532E1F910F91FF90C1
:105D4000EF900895EF92FF920F931F937C010E94B2
:105D50008F2E8C01C7010E94272D9C01200F311F1F
:105D6000C9011F910F91FF90EF9008950E94652D3A
:105D70000895EF92FF920F931F937C010E94B62E1D
:105D80008C01C7010E94272D9C01200F311FC901E2
:105D90001F910F91FF90EF90089508951F920F9219
:105DA0000FB60F9211242F933F934F938F939F938E
:105DB000EF93FF938091C80082FD1DC04091CE00FB
:105DC0002091B0063091B1062F5F3F4F2F73307096
:105DD0008091B2069091B3062817390771F0E091CF
:105DE000B006F091B106E059F94F40833093B10607
:105DF0002093B00602C08091CE00FF91EF919F9159
:105E00008F914F913F912F910F900FBE0F901F9048
:105E100018951F920F920FB60F9211242F933F9354
:105E20008F939F93EF93FF932091F4063091F506A3
:105E30008091F6069091F7062817390731F4809182
:105E4000C9008F7D8093C90014C0E091F606F091DF
:105E5000F706EC54F94F20818091F6069091F706F1
:105E600001968F7390709093F7068093F6062093B7
:105E7000CE00FF91EF919F918F913F912F910F90C5
:105E80000FBE0F901F9018958F929F92AF92BF9266
:105E9000CF92DF92EF92FF920F931F93DF93CF93F6
:105EA000CDB7DEB7FC011382128288EE93E0A0E04A
:105EB000B0E084839583A683B78389E094E09183DF
:105EC00080837587648757874687318B208B138B38
:105ED000028BF58AE48AD78AC68AB18EA08E938E09
:105EE000828E8F85848F8889858F8989868F8A891C
:105EF000878F8B8980A3CF91DF911F910F91FF90A6
:105F0000EF90DF90CF90BF90AF909F908F900895CB
:105F1000AF92BF92DF92EF92FF920F931F93CF93B6
:105F2000DF93EC017A018B01DD24403081EE5807CC
:105F300080E0680780E0780711F0DD24D39491E0D9
:105F4000A92EB12CEC89FD89DD2069F0C50108A0DE
:105F500002C0880F991F0A94E2F7808360E079E01D
:105F60008DE390E005C0108260E874E88EE190E077
:105F7000A80197010E94D135215030404040504047
:105F8000569547953795279580E12030380720F0C2
:105F9000DD2011F0DD24D6CFE889F9893083EA8944
:105FA000FB89208319A2EE89FF89408121E030E03E
:105FB000C9010C8C02C0880F991F0A94E2F7482B84
:105FC0004083EE89FF894081C9010D8C02C0880F92
:105FD000991F0A94E2F7482B4083EE89FF8940819C
:105FE000C9010E8C02C0880F991F0A94E2F7482B52
:105FF0004083EE89FF8980810F8C02C0220F331FFE
:106000000A94E2F7209528232083DF91CF911F91F6
:106010000F91FF90EF90DF90BF90AF900895DC015B
:106020001C96ED91FC911D97E05CFF4F2191319101
:1060300080819181281B390B2F733070C90108951D
:1060400088EF96E00E940F30892B11F00E94CD2E30
:106050000895DC011C96ED91FC911D97E05CFF4FCB
:1060600020813181E054F040DF01AE5BBF4F8D9164
:106070009C9111972817390719F42FEF3FEF07C0AC
:106080008D919C91E80FF91F8081282F30E0C90184
:106090000895DC011C96ED91FC911D97E05CFF4F8B
:1060A00020813181E054F040DF01AE5BBF4F8D9124
:1060B0009C9111972817390719F42FEF3FEF10C063
:1060C0008D919C911197E80FF91F20818D919C91E2
:1060D000119701968F73907011969C938E9330E078
:1060E000C9010895DC0191968C919197882339F02C
:1060F0005496ED91FC915597808186FFF9CF91964A
:106100001C920895CF93DF93EC01EE85FF85E05C50
:10611000FF4F20813181E054F0402F5F3F4F2F73BC
:106120003070DF01AE5BBF4F8D919C9111972817A6
:106130003907D1F3E05CFF4F80819181E054F0405A
:10614000E80FF91F6083EE85FF85E05CFF4F318328
:106150002083EE89FF89208181E090E00F8C02C0CE
:10616000880F991F0A94E2F7282B208381E089A3E6
:10617000EC89FD8980818064808381E090E0DF91FB
:10618000CF9108958F929F92AF92BF92CF92DF925C
:10619000EF92FF920F931F9300D000D00F92EDB7B4
:1061A000FEB7319684E0ADB7BEB711968C9383E00D
:1061B000818387E0828385E0838381E0848388EF25
:1061C00096E060E776E044EB56E02DEC30E00CEC36
:1061D00010E0B8ECEB2EF12CA9ECCA2ED12CFAEC85
:1061E000AF2EB12CEEEC8E2E912C0E94442F0F90EE
:1061F0000F900F900F900F901F910F91FF90EF90C5
:10620000DF90CF90BF90AF909F908F900895CF93E5
:10621000DF930E94762A82E297E00E94FE310E947C
:10622000C728C0E2D0E30E94F8142097E1F30E944F
:106230002030F9CFFC0104C08091F10081936150BE
:106240006623D1F7289884E680931B0708959FB7AB
:10625000F89487708093E9008091F2009FBF0895C1
:10626000282F80911C078823C1F057FF1AC015C042
:10627000289890931B078091F1008193E217F30710
:10628000B9F74115510539F08091F200882319F4CE
:106290008BE68093E800AFBF02C04FEF5FEFCA010B
:1062A0000895AFB7F89427702093E9008091F20029
:1062B000282F30E0241735070CF4A901FB019B01BE
:1062C000240F311D94E6DACFDF93CF930F92CDB731
:1062D000DEB7BE016F5F7F4F41E050E00E9430317A
:1062E000019719F02FEF3FEF03C08981282F30E08D
:1062F000C9010F90CF91DF9108952FB7F89487705F
:106300008093E9008091E80085FD02C090E004C020
:106310008091F20090E4981B2FBF892F089510926E
:10632000E90010921E0710921D079093200780939A
:106330001F070895FF920F931F93F82E142F052F18
:1063400040911F0750912007212F302FC901DC01F8
:10635000FB016EEF29C0F7FE02C0949101C090814D
:1063600020911D0730911E0724173507ACF480914A
:10637000E8008570E1F38091E80082FF03C02FEF11
:106380003FEF17C09093F100C90101968F73907091
:10639000892B11F46093E8002F5F3F4F30931E0765
:1063A00020931D07119731961097A9F6812F902FF2
:1063B0009C01C9011F910F91FF9008950F931F93A6
:1063C0009C01162F072F8091E80082FFFCCFC901A6
:1063D000612F0E941A318BEF8093E800812F902F5C
:1063E0001F910F9108958093E9008091F200882316
:1063F00019F08AE38093E8000895089510921C072D
:1064000081E08093D70080EA8093D80082E189BD43
:1064100009B400FEFDCF61E070E080E090E00E94F2
:10642000502A80E98093D8008CE08093E20010929B
:10643000E000559A209A08956F927F928F929F92D2
:10644000AF92BF92CF92DF92EF92FF920F931F9382
:10645000CF93DF93E82E942E852E80911C078823FE
:1064600009F18B01242F352FC901EC016AEFF62EBB
:1064700057E0752E7E208E2D90E040E2A42EB12CA8
:10648000A822B9223AE3632E20E4C22ED12CC822DE
:10649000D9224CC08E2D0E947D31282F882361F493
:1064A000FA9419F42FEF3FEF4CC061E070E080E008
:1064B00090E00E94502A3AC090E0C817D9070CF427
:1064C0002C2FC21BD1094FB7F8947092E900A11488
:1064D000B10421F406C01092F10021502223D9F713
:1064E00019C0E7FC03C0F801922F10C0C801322F79
:1064F00006C0FC010196E491E093F1003150332392
:10650000C1F706C081918093F10091509923D1F792
:10651000020F111D8091E80085FF05C0209729F426
:10652000C114D10411F06092E8004FBF209709F028
:10653000B1CF5D9884E680931A07292D382DC901C3
:106540009C01C901DF91CF911F910F91FF90EF90B6
:10655000DF90CF90BF90AF909F908F907F906F9083
:1065600008951F920F920FB60F9211242F933F930D
:106570004F935F936F937F938F939F93AF93BF934B
:10658000EF93FF938091E1001092E100982F93FF29
:106590000FC01092E90081E08093EB001092EC00B4
:1065A00082E38093ED0010921C0788E08093F00056
:1065B00092FF28C083E00E94F33182E00E942731DD
:1065C000882321F082E696E00E944A2C80911A07E7
:1065D000882351F080911A07815080931A07809187
:1065E0001A07882309F45D9A80911B07882351F0CC
:1065F00080911B07815080931B0780911B07882384
:1066000009F4289AFF91EF91BF91AF919F918F91DB
:106610007F916F915F914F913F912F910F900FBE9E
:106620000F901F9018950F931F93DF93CF930F92A6
:10663000CDB7DEB719828E010F5F1F4FC8010E94D0
:10664000702CC8010E949335898190E00F90CF9102
:10665000DF911F910F9108951F920F920FB60F9225
:106660001124CF92DF92EF92FF920F932F933F93DB
:106670004F935F936F937F938F939F93AF93BF934A
:10668000EF93FF93DF93CF93CDB7DEB76197DEBF74
:10669000CDBF1092E9008091E80083FFEBC0CE01EE
:1066A000019668E00E941A3182EF8093E800998198
:1066B00097FF05C08091E80080FFFCCF03C08EEFFC
:1066C0008093E800292F30E0C90180769070892BF3
:1066D00009F0B1C08A81882329F41092F100109248
:1066E000F100BDC0813009F4BAC0833009F4B7C0ED
:1066F000853049F48091E80080FFFCCF8B81806871
:106700008093E300ACC0863009F06BC00C81EF8051
:10671000F884023071F580E090E00E948F310E9491
:10672000133399E079E0C72ED12CCC0EDD1EF60193
:10673000292F11922A95E9F799870A8791E09E8778
:1067400090E8988B9AEF998B20911D0730911E0746
:10675000275F3F4F3C872B878D87C7010E948F3172
:1067600080E0B60149E050E00E949A310E94133364
:1067700076C0C7010E948F31023241F482E290E07C
:106780000E948B35892B09F46EC069C0013079F401
:106790008F819885089719F481E080932107809173
:1067A0002107882309F063C0ECEBFCE013C0033041
:1067B00009F059C08B81882319F4EEE7FCE00AC088
:1067C000823019F4E2E8FCE005C0813009F04BC0EA
:1067D000E4EAFCE0449180E8BF0150E00E949A3175
:1067E0003EC0873009F43FC0883021F481E08093B7
:1067F000F10035C0893099F523703070232B99F55D
:10680000E1EEFCE091E031E026E39093E900309383
:10681000EB0084918093EC002093ED009F5F319614
:10682000953099F78EE78093EA001092EA008B8109
:1068300080931C0714C08F8198850E948F318D81B1
:10684000882329F4CE0101960E947C2C06C0823058
:1068500051F4CE0101960E945534882321F08EEF29
:106860008093E80007C081E28093EB0003C0EEEC68
:10687000FCE0B0CF6196DEBFCDBFCF91DF91FF913D
:10688000EF91BF91AF919F918F917F916F915F91A8
:106890004F913F912F910F91FF90EF90DF90CF900C
:1068A0000F900FBE0F901F901895FC019181808171
:1068B000813A31F4913089F080E0933089F40DC051
:1068C000813269F49B3021F482818093B30305C047
:1068D0009A3029F482818093B40381E0089580E0A6
:1068E0000895FC0110820895FC011382128289E14F
:1068F00094E0918380830895EF92FF920F931F930A
:106900008C01E62EDC01ED91FC910480F581E02DF7
:106910000995F82ED801ED91FC910680F781E02DC4
:10692000C8016E2D09958F2D90E01F910F91FF905A
:10693000EF90089583E297E00E94713484E297E03B
:106940000E9474340895EF92FF920F931F93DF9388
:10695000CF930F92CDB7DEB789838B017A0184E0A4
:10696000BE016F5F7F4F41E050E00E941C3284E423
:10697000B801A7010E941C320F90CF91DF911F91A7
:106980000F91FF90EF90089582E048E050E00E9460
:10699000A3340895FC011682178210861186128690
:1069A000138614823496BF010E94C4340895DC011A
:1069B000683810F0685829C0E62FF0E067FF13C070
:1069C000E058F04081E090E002C0880F991FEA95FE
:1069D000E2F7809514962C911497282314962C9303
:1069E000149760E012C0ED59F24F6491662319F4D8
:1069F00020E030E01DC067FF08C014968C9114970A
:106A00008D7F14968C9314976F77FD0190E0662329
:106A100021F08681861709F416829F5F31969630A1
:106A2000B1F7CD011496BD010E94C43421E030E0DD
:106A3000C9010895CF93DF93DC01683810F06858DE
:106A400025C0E62FF0E067FF12C0E058F04081E07B
:106A500090E002C0880F991FEA95E2F714962C91F6
:106A60001497282B14962C93149760E00FC0ED59BF
:106A7000F24F64916623D9F167FF08C014968C9198
:106A80001497826014968C9314976F7716968C9156
:106A900016978617A9F117968C911797861781F18B
:106AA00018968C911897861759F119968C91199709
:106AB000861731F11A968C911A97861709F11B9651
:106AC0008C911B978617E1F0ED01E0E0F0E09E2F3E
:106AD0008E81882321F4EA0FFB1F668306C09F5F27
:106AE00031962196E630F10591F7963049F481E030
:106AF00090E013969C938E93129720E030E007C0AD
:106B0000CD011496BD010E94C43421E030E0C901DA
:106B1000DF91CF91089580E865EE7CE045E650E096
:106B20000E949A310895FC0180818F5F808380E804
:106B30006AE47DE049E150E00E949A310895629F45
:106B4000D001739FF001829FE00DF11D649FE00D65
:106B5000F11D929FF00D839FF00D749FF00D659FC6
:106B6000F00D9927729FB00DE11DF91F639FB00DC5
:106B7000E11DF91FBD01CF011124089597FB092ED6
:106B800007260AD077FD04D049D006D000201AF499
:106B9000709561957F4F0895F6F7909581959F4F79
:106BA0000895A1E21A2EAA1BBB1BFD010DC0AA1F4E
:106BB000BB1FEE1FFF1FA217B307E407F50720F066
:106BC000A21BB30BE40BF50B661F771F881F991FE1
:106BD0001A9469F760957095809590959B01AC012A
:106BE000BD01CF01089597FB092E05260ED057FD54
:106BF00004D0D7DF0AD0001C38F45095409530956A
:106C000021953F4F4F4F5F4F0895F6F79095809530
:106C1000709561957F4F8F4F9F4F0895AA1BBB1BA7
:106C200051E107C0AA1FBB1FA617B70710F0A61B8C
:106C3000B70B881F991F5A95A9F780959095BC01AD
:106C4000CD010895EE0FFF1F0590F491E02D0994FA
:106C5000911106C0803219F089508550D0F70895FF
:106C60009927882708952F923F924F925F926F92B3
:106C70007F928F929F92AF92BF92CF92DF92EF92CC
:106C8000FF920F931F93CF93DF93CDB7DEB7CA1B4D
:106C9000DB0B0FB6F894DEBF0FBECDBF09942A8878
:106CA000398848885F846E847D848C849B84AA8420
:106CB000B984C884DF80EE80FD800C811B81AA81AD
:106CC000B981CE0FD11D0FB6F894DEBF0FBECDBF78
:086CD000ED010895F894FFCFD7
:106CD8004E6F005965730054582074696D656F755F
:106CE8007421006D6F64756C65206C6F636B6564EF
:106CF8003F00486F70206368616E6E656C200020ED
:106D080040200053004E2F4100386368002C002CAF
:106D1800205B005D20280029004E4F5420454E413D
:106D2800424C45440053656E64696E672073657410
:106D380074696E677320746F2052580A0052657325
:106D4800657474696E672073657474696E677320FF
:106D58006F6E2052580A0041626F72746564206534
:106D6800646974730A00696E76616C69642073657E
:106D78006C656374696F6E000D0A496E76616C69A3
:106D88006420696E707574202D2064697363617264
:106D98006465642107007363616E6E6572206D6FB0
:106DA80064650053657474696E67732073617665F2
:106DB8006420746F20454550524F4D0A0052657645
:106DC80065727465642073657474696E6773206690
:106DD800726F6D20454550524F4D0A004C6F6164EB
:106DE800656420666163746F727920646566617595
:106DF8006C74730A004B657920616E642063686166
:106E08006E6E656C732072616E646F6D697A65640D
:106E18000A004E65772070726F66696C653A004C9F
:106E28006F616465642073657474696E6773206646
:106E3800726F6D20454550524F4D0A0045455052DE
:106E48004F4D2064617461206E6F742076616C69A7
:106E5800642C207265696E6974696E670A00456EF4
:106E6800746572696E672062696E64696E67206D09
:106E78006F64650A004F70656E4C52536E672054FC
:106E880058207374617274696E672000206F6E20D9
:106E98004857200050504D00525353490053444125
:106EA8000053434C00525844005458440041494E42
:106EB800004C424545500053504B54524D005342EC
:106EC80055530053554D44004C4C494E4400003432
:106ED8002B34003800382B340031320031322B3457
:106EE8000031360001000000C01200001A400AA15B
:106EF800204EA5001B1E27522C233080250000059C
:106F0800400AA1204EA50020244EA52C2330004B7A
:106F1800000006400AD0009D49007B289D492C238B
:106F28003000E1000005400A4501D7DC03B81E0E19
:106F3800BF00232E48E801008A400A600155550227
:106F4800AD1E20000023C88025000005400AA120AE
:106F58004EA50020244EA52C23300002000200027A
:106F68000002000200020002000200020002000209
:106F780000020002000200020002FF00E10000001F
:106F88000000000101C402C802CD02D102D502D915
:106F980002DD02E102E702EE02F302F802FE02FE5F
:106FA80002FE02FE023501FF020303050309030C7A
:106FB800031103350100070B0C10111500160A13F5
:106FC800223129000000001E2CD22CBD2BE42BCB33
:106FD8002B462C4A2C000000008230D22C0F30495E
:106FE8003029307230000000007C34D22C1A35D79A
:046FF80034CA340063
:00000001FF
